S024000062696E2F6F70656E62746C5F6F6C696D65785F73746D3332653430372E737265639F
S31508000000642D0020417400082D7400082D74000822
S315080000102D7400082D7400082D7400082D7400082E
S315080000202D7400082D7400082D7400082D7400081E
S315080000302D7400082D7400082D7400082D7400080E
S315080000402D7400082D7400082D7400082D740008FE
S315080000502D7400082D7400082D7400082D740008EE
S315080000602D7400082D7400082D7400082D740008DE
S315080000702D7400082D7400082D7400082D740008CE
S315080000802D7400082D7400082D7400082D740008BE
S315080000902D7400082D7400082D7400082D740008AE
S315080000A02D7400082D7400082D7400082D7400089E
S315080000B02D7400082D7400082D7400082D7400088E
S315080000C02D7400082D7400082D7400082D7400087E
S315080000D02D7400082D7400082D7400082D7400086E
S315080000E02D7400082D7400082D7400082D7400085E
S315080000F02D7400082D7400082D7400082D7400084E
S315080001002D7400082D7400082D7400082D7400083D
S315080001102D7400082D7400082D7400082D7400082D
S315080001202D7400082D7400082D7400082D7400081D
S315080001302D7400082D7400082D7400082D7400080D
S315080001402D7400082D7400082D7400082D740008FD
S315080001502D7400082D7400082D7400082D740008ED
S315080001602D7400082D7400082D7400082D740008DD
S315080001702D7400082D7400082D7400082D740008CD
S315080001802D7400082D74000810B572B61748184962
S31508000190016018498D4640F20002C2F2000240F2A0
S315080001A02003C2F200039A4210D2131D0E4CE41A21
S315080001B024F0030404340023104647F69871C0F669
S315080001C000015A581A500433A342FAD10A480B4977
S315080001D04FF000028842B8BF40F8042BFADB05F05E
S315080001E04BFD00F0AFF810BD2300002008ED00E03D
S315080001F000000008642D00208000002064250020EF
S3150800020000B589B0002300930193029303930493E6
S3150800021005930693079347F2E850C0F6000069462F
S3150800022004F07CF848B9009B002043B19DF808000B
S3150800023080F01000C0F3001001E00020FFE709B0CD
S315080002405DF804FB47F2E850C0F60000704700BFAF
S3150800025008B540F28000C2F20000002380F824327C
S3150800026047F20861C0F600010A2203F0B5FC30B96E
S3150800027040F28003C2F20003012283F8242208BD5B
S3150800028038B540F28003C2F2000393F82432012BFA
S3150800029005D140F28000C2F2000003F069FF4FF476
S315080002A0A054C4F2010440252046294602F020F94C
S315080002B00028F9D047F2E850C0F6000004F054F8D8
S315080002C038BD00BF08B540F28003C2F2000393F8B8
S315080002D02432012B05D140F28000C2F2000003F05F
S315080002E047FF08BD70B5064640F28003C2F2000318
S315080002F093F82432012B10D140F28001C2F200019A
S3150800030004F0D2F8002808DA40F28000C2F20000B1
S31508000310002380F8243203F02BFF317889B14FF49B
S31508000320A054C4F201048025204602F0D9F82046DC
S31508000330294602F0DDF80028F9D016F8011F002931
S31508000340F2D170BD80B582B072B602F0D7F820201F
S31508000350012101F06BFF0420012101F043FF4FF456
S315080003600065C4F2020528460621082201F0B8FEF7
S3150800037028460721082201F0B3FE00278DF80670EB
S3150800038001268DF8076002248DF804404023009367
S315080003908DF805402846694601F054FE8DF804405C
S315080003A0802300932846694601F04CFE20463146D4
S315080003B001F018FF4FF48065C4F2020528460521AE
S315080003C0092201F08DFE28460621092201F088FE41
S315080003D0602300938DF804408DF805408DF806706B
S315080003E08DF807602846694601F02CFE4FF0C0607C
S315080003F0314601F009FF05F07DFB05F089FBFCE7B6
S3150800040008B54FF43053C4F201035B6B13F0450F84
S3150800041007D14FF43052C4F20102536B13F0450F63
S31508000420FBD013F0040F04D0042001F0CFFF032003
S3150800043008BD13F0010F04D0012001F0C7FF012009
S3150800044008BD40F2FF5001F0C1FF002008BD00BF03
S3150800045010B504464FF43053C4F201035B6B13F036
S31508000460450F07D14FF43052C4F20102536B13F013
S31508000470450FFBD013F0040F04D0042001F0A6FFAB
S31508000480032010BD13F0010F04D0012001F09EFFD8
S31508000490012010BD01F052FFA04249D140F2FF50A1
S315080004A001F094FF002001F051FF4EF20803CFF649
S315080004B0FF530340002B3DD000283DDB10F0804F52
S315080004C03CD110F0005F3BD110F0805F3AD110F0BC
S315080004D0006F39D110F0806F38D110F0807F37D196
S315080004E010F4000F36D110F4800F35D110F4001F28
S315080004F034D110F4801F33D110F4002F32D110F408
S31508000500802F31D110F4003F30D110F4803F2FD125
S3150800051010F4004F2ED110F4804F2DD110F4005F47
S315080005202CD100F00800002814BF1A20002010BDA6
S31508000530102010BD002010BD1C2010BD092010BDC4
S315080005400A2010BD0B2010BD0C2010BD0D2010BDBB
S315080005500E2010BD0F2010BD102010BD112010BD9B
S31508000560122010BD132010BD142010BD152010BD7B
S31508000570162010BD172010BD182010BD192010BD5B
S315080005802DE9F04182B00446002001F0DFFE10F0AC
S31508000590007F18BF0E2040F01781002200920192BA
S315080005A040F26030C2F20000082101601025456063
S315080005B040218160C2604FF48062026101F0A6FEAC
S315080005C02846FFF745FF002840F0FC8040F26030DF
S315080005D0C2F2000040F20432C2F200021268AA40D7
S315080005E0026037254560402282600022C2604FF4CF
S315080005F08062026101F08AFE2846FFF729FF00287B
S3150800060040F0E18040F2AC20C2F200004FF0FF3328
S31508000610036008234360302383600223C3600025F8
S3150800062005610123436101F09FFE40F26030C2F28A
S31508000630000005603326466040228260C5604FF49C
S315080006408062026101F062FE3046FFF701FF002872
S3150800065040F0BA80ADF104084FF43055C4F20105F4
S3150800066040F22A664FF4001707E0384601F0A4FE68
S3150800067018B101F091FE48F8040F6B6B3342F4D0C1
S31508000680082001F099FE20B1082001F09FFE042001
S315080006909AE0022001F090FE20B1022001F096FEB9
S315080006A0022091E0202001F087FE20B1202001F0F1
S315080006B08DFE062088E04FF4007001F07DFE28B11B
S315080006C04FF4007001F082FE07207DE040F2FF50F3
S315080006D001F07CFE009A130643EA126302F47F4196
S315080006E043EA012302F47F0243EA1223012C34D1A0
S315080006F013F4802F08BF252066D040F26030C2F27E
S31508000700000040F20432C2F20002126812040260CB
S3150800071037244460402282600022C2604FF480621F
S31508000720026101F0F3FD2046FFF792FE002847D14B
S3150800073040F26030C2F200000222026006244460E1
S31508000740402282600022C2604FF48062026101F09A
S31508000750DDFD2046FFF77CFE36E013F4803F08BF38
S31508000760252031D040F26030C2F2000040F2043257
S31508000770C2F2000212681204026037244460402262
S3150800078082600022C2604FF48062026101F0BEFD01
S315080007902046FFF75DFEA0B940F26030C2F20000C5
S315080007A0002202600624446040218160C2604FF442
S315080007B08062026101F0AAFD2046FFF749FE03E0C8
S315080007C002E001E000E0FFE702B0BDE8F08100BF0B
S315080007D000B583B001238DF807304FF40060C4F2EA
S315080007E002004FF4006101F075FC10B900238DF882
S315080007F007309DF8070003B05DF804FB2DE9F047C4
S3150800080082B000248DF8074040F2EC20C2F20000C6
S3150800081076230375046044608460C460046101F053
S3150800082047FD032001F064FD012001F05BFD40F265
S315080008306030C2F20000046044608460C4604FF413
S315080008408063036101F062FD4FF48034802501E086
S31508000850013C0CD0284601F0AFFD0028F8D0032350
S315080008603CB140F2FF5001F0B1FD002301E0032343
S31508000870FFE78DF807309DF8073013F0FF0F03D018
S315080008809DF80700C0B2F5E040F26030C2F2000001
S315080008904FF4D57303600823436040238360002325
S315080008A0C3604FF48063036101F030FD4FF43053A9
S315080008B0C4F201035A6B12F0450F0ED14FF4803380
S315080008C04FF43051C4F20101013B4A6B12F0450F57
S315080008D002D1002BF8D103E013B112F0040F04D0B3
S315080008E0042001F073FD032309E012F0400F08BF4E
S315080008F0002304D0402001F069FD0023FFE78DF8AE
S3150800090007309DF8073013F0FF0F08D140F2D423C3
S31508000910C2F2000301221A604FF0804514E040F24B
S315080009206030C2F20000002505603724446040228A
S315080009308260C5604FF48062026101F0E7FC2046E0
S31508000940FFF786FD8DF8070040F26030C2F200001E
S31508000950002202603724446040218160C2604FF45F
S315080009608062026101F0D2FC2046FFF771FD8DF826
S3150800097007009DF8073013F0FF0F78D1002740F2E3
S315080009806034C2F20004B846B94645F0004545F45D
S31508000990801A4FF43055C4F20105C4F80090372682
S315080009A066604023A360C4F80C904FF4806323610B
S315080009B0204601F0ABFC3046FFF74AFD8DF80700EC
S315080009C09DF8073013F0FF0F03D09DF80700C0B25B
S315080009D050E0C4F800A0292363604023A360C4F84C
S315080009E00C804FF480632361204601F08FFC6B6B0B
S315080009F013F0450F03D16B6B13F0450FFBD013F0C3
S31508000A00040F04D0042001F0E1FC032304E040F2C3
S31508000A10FF5001F0DBFC43468DF807309DF80730A0
S31508000A2013F0FF0F03D09DF80700C0B222E040463E
S31508000A3001F08CFC013701464FF6FE73C043C00F28
S31508000A409F4288BF00200028A7D19F4206D91B23B2
S31508000A508DF807309DF80700C0B20BE011F0804F03
S31508000A601FBF40F2D423C2F2000302221A609DF887
S31508000A700700C0B202B0BDE8F08700BF38B501F084
S31508000A803DFC002800F0BC8040F2D423C2F20003EB
S31508000A901B68042B00F0B68040F26030C2F20000FA
S31508000AA00023036002224260C0228260C3604FF4C2
S31508000AB08063036101F02AFCFFF7A2FC002840F0DE
S31508000AC0A38001F043FC40F2D824C2F2000420605F
S31508000AD0042001F03BFC6060082001F037FCA060B0
S31508000AE00C2001F033FCE06040F2D423C2F200038C
S31508000AF01B68062B18BF022B88BF01224AD840F272
S31508000B006030C2F2000000230360032242604022E4
S31508000B108260C3604FF48063036101F0F7FB4FF412
S31508000B203053C4F201035B6B13F0450F07D14FF442
S31508000B303052C4F20102536B13F0450FFBD013F089
S31508000B40040F04D0042001F041FC032038BD13F043
S31508000B50010F04D0012001F039FC012038BD01F055
S31508000B60EDFB032854D140F2FF5001F02FFC002082
S31508000B7001F0ECFB10F4604F08BF020C0AD010F429
S31508000B80005F47D110F4804F46D110F4004F45D18D
S31508000B900122FFE740F2D423C2F200031B68042BAC
S31508000BA033D040F20433C2F200031A6040F26030D8
S31508000BB0C2F200001204026009234360C023836066
S31508000BC00023C3604FF48063036101F09FFBFFF7C6
S31508000BD017FC0546D8B901F0B9FB40F2C424C2F2A5
S31508000BE000042060042001F0B1FB6060082001F0D9
S31508000BF0ADFBA0600C2001F0A9FBE060284638BDDB
S31508000C00252038BD002038BD38BD002038BD38BD88
S31508000C10102038BD132038BD102038BD0F2038BD30
S31508000C20F0B4014640F2D423C2F200031C6880F8EF
S31508000C30564040F20433C2F200031B68A0F8543051
S31508000C4040F2C423C2F200031A68150EE8B28609F8
S31508000C500E70C5F383054D7000F003008870C2F36B
S31508000C600740C870C2F307200871D2B24A715B68A0
S31508000C701A0E1201CA80C3F30742C88880B240EA36
S31508000C801210C88002F00F020A72C3F30720C209C5
S31508000C904A72C0F380128A72C0F34012CA72C0F355
S31508000CA000120A7300224A73012C42D800F003008E
S31508000CB0800208610A69DBB242EA83030B6140F2EB
S31508000CC0C423C2F200039868020ED3B20C6944EA40
S31508000CD093140C61C2F3C2020A7503F007034B753D
S31508000CE0C0F307435A098A75C3F38202CA7503F02B
S31508000CF003035B000B76C0F307200B7E43EAD01391
S31508000D000B760F690A7E0E7AF6B2012303FA06F607
S31508000D100E65023203FA02F2D517A2FB062306FB7A
S31508000D2005337E1CA2FB064506FB0355C1E91245A1
S31508000D3024E0022C22D103F03F031B040B6140F28E
S31508000D40C423C2F2000398680B69020E43EA022321
S31508000D500B610B69C0F3074213430B61C0F307200D
S31508000D600A690023013243F10003DB0443EA5233E4
S31508000D70D2048A64CB644FF400730B65C0F3801306
S31508000D804B7600F03F004000887640F2C423C2F25A
S31508000D9000031A7A887E40EAD210887602F07F022B
S31508000DA0CA76DA68130ED8B2C4090C77C3F34114AD
S31508000DB04C77C3F382038B7700F003008000C87773
S31508000DC0C2F30743C87F40EA9310C877C3F34010BD
S31508000DD081F82000002081F8210003F0010381F842
S31508000DE02230C2F30723DC0981F82340C3F38014B9
S31508000DF081F82440C3F3401481F82540C3F3001456
S31508000E0081F82640C3F3810481F8274003F00303E1
S31508000E1081F82830C2F3460281F82920012481F896
S31508000E202A4040F2D823C2F200031A68150E81F848
S31508000E302C50C2F307452D02CD85CD8DADB2C2F338
S31508000E4007263543CD8512060A635A680D6B160EBA
S31508000E5045EA06450D630D6BC2F3074645EA0625C6
S31508000E600D630D6BC2F3072635430D63D2B281F8C5
S31508000E7034209A68150E81F83550C2F307452D06B9
S31508000E808D638D6BC2F3072645EA06458D638D6B28
S31508000E90D2B245EA02228A63DB688A6B42EA1362A7
S31508000EA08A63C3F3074291F83C5045EA121581F864
S31508000EB03C5002F00F021202CA87CA8F92B2C3F3DD
S31508000EC007252A43CA87C3F3460381F8403081F8C9
S31508000ED04140F0BC704700BF10B540F2D423C2F2BF
S31508000EE000031B68032B31D0022B31D8B0F5805F85
S31508000EF030D0B0F5006F15D10120FFF741FB04464D
S31508000F0050BB40F2EC20C2F20000002202750260DB
S31508000F10426082604FF40061C160026101F0C8F965
S31508000F20204610BD0020FFF72BFB0446A8B940F267
S31508000F30EC20C2F200000022027502604260826064
S31508000F40C260026101F0B4F9204610BD272010BD29
S31508000F50002010BD272010BD10BD10BD10B540F2F1
S31508000F606033C2F20003186007245C6040229A606E
S31508000F700022DA604FF480621A61184601F0C6F959
S31508000F802046FFF765FA10BD2DE9F04184B000262A
S31508000F908DF80F600C20012101F024F94FF400644C
S31508000FA0C4F20204204608210C2201F099F82046D2
S31508000FB009210C2201F094F820460A210C2201F09E
S31508000FC08FF820460B210C2201F08AF820460C21C6
S31508000FD00A4601F085F84FF44067C4F2020738461E
S31508000FE002210C2201F07CF84FF47063019301256D
S31508000FF08DF809504FF002088DF808808DF80A60C0
S315080010008DF80B50204601A901F01CF80423019322
S3150800101038460DEB030101F015F84FF480530193A0
S315080010208DF80B60204601A901F00CF84FF4006713
S3150800103001978DF808808DF80B60204601A901F00C
S3150800104001F83846294601F0F1F84FF480002946A0
S3150800105001F0C8F801F020F9FFF7D0FB8DF80F0072
S315080010609DF80F3013F0FF0F03D09DF80F00C0B2A4
S3150800107040E0FFF703FD8DF80F009DF80F3013F0E1
S31508001080FF0F03D09DF80F00C0B233E040F2EC200A
S31508001090C2F2000000230375036043608360C360E7
S315080010A0036101F005F940F20830C2F20000FFF7CB
S315080010B0B7FD8DF80F009DF80F3013F0FF0F0BD119
S315080010C040F20833C2F20003B3F8540000040021CA
S315080010D0FFF744FF8DF80F009DF80F3013F0FF0F50
S315080010E005D14FF40060FFF7F7FE8DF80F009DF865
S315080010F00F00C0B204B0BDE8F08100BF2DE9F84387
S3150800110007461646BDF8204040F2A822C2F2000261
S315080011100021117040F2E822C2F20002116040F28A
S315080011207430C2F2000001604FF43052C4F201027A
S31508001130D16240F2D421C2F200010A68022A02BF33
S31508001140760A46EAC3564FF40074A04640F2603069
S31508001150C2F200000460102242604022826000222F
S31508001160C2604FF48062026101F0D0F84FF4803417
S31508001170802501E0013C04D0284601F01DF900282D
S31508001180F8D01020FFF764F9002840F0868040F276
S31508001190AC20C2F200004FF0FF330360C0F80480B1
S315080011A0902383600223C360002505610123436100
S315080011B001F0DAF840F26030C2F20000066011244D
S315080011C0446040228260C5604FF48062026101F08B
S315080011D09DF82046FFF73CF9002860D14FF43055BA
S315080011E0C4F2010540F22A664FF400484FF00009A0
S315080011F00BE0404601F0E0F838B14C4601F0CCF877
S3150800120038510434202CF9D120376B6B3342F0D097
S31508001210082001F0D1F828B1082001F0D7F80420F9
S31508001220BDE8F883022001F0C7F828B1022001F0D2
S31508001230CDF80220BDE8F883202001F0BDF828B1DA
S31508001240202001F0C3F80620BDE8F8834FF40070AB
S3150800125001F0B2F84FF0FF344FF4001558B14FF4CF
S31508001260007001F0B3F80720BDE8F88301F094F8A0
S3150800127047F8040B013C284601F09EF808B1002CFB
S31508001280F4D140F2FF5001F0A1F840F20003C2F297
S31508001290000300201860BDE8F883BDE8F883BDE8C0
S315080012A0F88300BF2DE9F84F80461446BDF828207C
S315080012B040F2A820C2F200000021017040F2E820A6
S315080012C0C2F20000016040F27430C2F20000016010
S315080012D04FF43050C4F20100C16240F2D421C2F288
S315080012E000010968022902BF640A44EAC3544FF49C
S315080012F00072164640F26030C2F200000260102505
S315080013004560402282600022C2604FF4806202611A
S3150800131000F0FCFF2846FFF79BF8002840F08B807A
S3150800132040F26030C2F20000046018244460402293
S3150800133082600022C2604FF48062026100F0E6FF1C
S315080013402046FFF785F8002877D140F2AC20C2F294
S3150800135000004FF0FF33036046609023836000244B
S31508001360C46004610123436100F0FEFFA3464FF405
S315080013703054C4F2010440F21A654FF4804625E061
S31508001380304601F019F808B3CBF5007ABAF11F0F09
S3150800139010D85FEA9A0A19D0C146002759F8040BF3
S315080013A001F002F801375745F8D14FEA8A0AD044C6
S315080013B0D3440BE0002758F8070000F0F5FF043780
S315080013C0202FF8D108F120080BF1200B636B2B4274
S315080013D0D6D0082000F0F0FF28B1082000F0F6FF6C
S315080013E00420BDE8F88F022000F0E6FF28B10220AD
S315080013F000F0ECFF0220BDE8F88F102000F0DCFFBB
S3150800140028B1102000F0E2FF0520BDE8F88F4FF460
S31508001410007000F0D1FF30B14FF4007000F0D6FF35
S315080014200720BDE8F88F40F20003C2F2000300204F
S315080014301860BDE8F88FBDE8F88FBDE8F88F00BFE3
S3150800144038B50546F8B140F26030C2F2000040F205
S315080014500432C2F200021268120402600D244460CB
S31508001460402282600022C2604FF48062026100F06E
S315080014704DFF2046FEF7ECFF044630B900F066FF44
S315080014802860204638BD262038BD38BD00B583B053
S3150800149000230193FFF79CF9012818BFFF2008D104
S315080014A001A8FFF7CDFF18B90198C0F3432000E063
S315080014B0FF2003B05DF804FB08B5FFF7E7FF042833
S315080014C004D0FF2814BF0120022008BD002008BD53
S315080014D000B597B0FFF758FD60B940F20403C2F2B1
S315080014E000031A7802F0FE021A706846FFF798FBA6
S315080014F0002006E040F20403C2F2000301221A703B
S31508001500032017B05DF804FB08B540F20403C2F2E5
S31508001510000301221A7050B9FFF7CEFF38B940F21E
S315080015200403C2F200031A7802F0FE021A7040F2AF
S315080015300403C2F20003187808BD00BF2DE9F04382
S31508001540ADF5037D88461746D0B11CE0013BDCB2F9
S315080015504FF000094FF40075E619009502A87202CB
S315080015604B46FFF7CBFD80B9FFF7A6FF0128FBD056
S3150800157008EB442002A92A4605F092FF4CB906E07A
S3150800158001204BB1E2E7012006E0012004E000203B
S3150800159002E0013CE4B2DFE70DF5037DBDE8F08328
S315080015A02DE9F043ADF5037D0F469046F0B120E0F6
S315080015B0013BDCB24FF400754FF0000902A807EBB7
S315080015C044212A4605F06CFF04EB0806009502A89C
S315080015D072024B46FFF766FE052818BF00280AD197
S315080015E0FFF76AFF0128FBD04CB906E001204BB192
S315080015F0DEE7012006E0012004E0002002E0013CCD
S31508001600E4B2DBE70DF5037DBDE8F08310B596B0CF
S31508001610144640F20403C2F200031B7813F0010FCC
S3150800162018BF032021D103291AD8DFE801F00204E4
S315080016301015002019E0A8B96846FFF7F1FA129BC1
S315080016405B0A139A43EAC253236000200DE04FF465
S3150800165000731380002008E030B92023136004E0EB
S31508001660042002E0002000E0002016B010BD00BFF4
S315080016700020C4F2AA20704708B54FF00070012177
S3150800168000F0E6FD4FF00070002100F0E1FD08BD16
S315080016900023036043608360C36003614361836121
S315080016A0C361036243628362C36203634363836302
S315080016B0C36340220264202242648364C3640365D0
S315080016C043658365C3650366802242668366C3668F
S315080016D0036743678367C3674FF08062C0F880205B
S315080016E04FF00072C0F884204FF08071C0F888105F
S315080016F04FF40011C0F88C10C0F89030C0F8943040
S31508001700C0F89830C0F89C30C0F8A030C0F8A420C3
S31508001710C0F8A8304FF40032C0F8AC204FF48072FD
S31508001720C0F8B020C0F8B430C0F8B830704700BF71
S3150800173082B0002301934FF40043C4F202031A69EE
S3150800174002F01C02890101F4F8610A43C00281B261
S315080017500A4342F001021A614FF40042C4F202023F
S315080017604FF6FE71C0F20401019B01330193136920
S3150800177013F0010F02D0019B8B42F5D9019A4FF65F
S31508001780FF73C0F204039A421FBF4FF40043C4F22A
S315080017900203586980B208BF002002B0704700BF34
S315080017A010B483B0002301934FF40043C4F202033C
S315080017B01C6904F01C0444F00304890101F4F8616F
S315080017C00C43C00281B20C435A611C614FF40042BB
S315080017D0C4F202024FF6FE71C0F20401019B013306
S315080017E00193136913F0010F02D0019B8B42F5D9BF
S315080017F001984FF6FF73C0F20403C01A18BF012000
S3150800180003B05DF8044B7047F0B587B004460D4643
S315080018100023059300934FF40043C4F202031E69A4
S3150800182026F01C0601A800F06FFC02994FF45343FA
S31508001830CFF6CE630B444EF2BF12C0F2E4029342D7
S3150800184098BF46F008061AD94FF24013CFF6E95367
S315080018500B4447F63F02C0F27D12934298BF46F00A
S315080018600C060CD94FF4F243CFF66C430B444FF4F5
S31508001870B442C0F26222934288BF46F004064FF48F
S315080018800043C4F202031E61284600214FF40042B9
S31508001890FFF786FF002800F00F814FF0806305935D
S315080018A0059B2BB1059B013B0593059B002BF9D1A5
S315080018B02368002B5ED001274FF6FE76C0F2040699
S315080018C0009B0133009328463946FFF731FF00F0A5
S315080018D0040083B213B9009BB342F1D9009A4FF6BC
S315080018E0FF73C0F204039A4208BF002000F0E980A3
S315080018F00021009128464FF48052FFF751FF002837
S3150800190000F0DC8001274FF6FE76C0F20406009B45
S315080019100133009328463946FFF70AFF00F02000F6
S3150800192080B210B9009BB342F1D9009A4FF6FF7303
S31508001930C0F204039A4208BF002000F0C2800023C8
S31508001940009328461021FFF7F3FE00F004039BB22C
S315080019501BB14FF40063236201E00023236200F009
S3150800196002039BB213B1002363611BE04FF480436B
S31508001970636117E06369226AD20842EA530228467D
S31508001980002192B2FFF70CFF002800F099806FF053
S315080019907F430593059B2BB1059B013B0593059B4F
S315080019A0002BF9D14FF40043C4F20203196848F238
S315080019B00F12CFF620720A40A06861680843E168F2
S315080019C008432169084361690843A1690843E16935
S315080019D00843216A0843616A0843A16A0843E16A21
S315080019E00843216B0843616B01430A431A60E16BA4
S315080019F0A26B1143226C1143626C1143A26C114312
S31508001A00E26C1143226D1143626D0A435A60A26D5E
S31508001A109A60E26DDA609869A16E626E1143E26EB1
S31508001A201143226F1143626F11434FF64172024010
S31508001A300A43216E42EA01419961E16FA26F0A43A6
S31508001A40DA6103F58053996943F62372CFF6DE020D
S31508001A500A40D4F88400D4F880100843D4F88810D3
S31508001A600843D4F88C100843D4F890100843D4F8E7
S31508001A7094100843D4F898100843D4F89C100843E7
S31508001A80D4F8A01001430A439A61D4F8A410D4F8F4
S31508001A90A820114341F40001D4F8AC201143D4F82E
S31508001AA0B0201143D4F8B8200A43D4F8B41042EA57
S31508001AB081021A60012004E0002002E0002000E014
S31508001AC0002007B0F0BD00BF40B14FF40043C4F298
S31508001AD002031A6842F008021A6070474FF400437E
S31508001AE0C4F202031A6822F008021A60704700BF9F
S31508001AF040B14FF40043C4F202031A6842F00402EC
S31508001B001A6070474FF40043C4F202031A6822F0C1
S31508001B1004021A60704700BF4FF41043C4F2020370
S31508001B201A6842F001021A60704700BF4FF410436A
S31508001B30C4F20203186800F0010070474FF410431E
S31508001B40C4F202039A6942F480129A61704700BF90
S31508001B5040B14FF41043C4F202039A6942F40052AA
S31508001B609A6170474FF41043C4F202039A6922F44B
S31508001B7000529A61704700BF40B14FF41043C4F257
S31508001B8002039A6942F002029A6170474FF41043C1
S31508001B90C4F202039A6922F002029A61704700BFF2
S31508001BA008B50120FFF790FFFFF7C8FF0120FFF7F0
S31508001BB09FFF0120FFF7CCFF0120FFF7DDFF08BDDF
S31508001BC02DE9F047B2B04FF0F050012100F00AFBC2
S31508001BD04720012100F006FB4FF48040012100F068
S31508001BE025FB012000F0F8FB8E23309300268DF8A4
S31508001BF0C66002248DF8C4408DF8C7608DF8C540CC
S31508001C003746C4F20207384630A900F01BFA3846B0
S31508001C1001210B2200F064FA384621460B2200F017
S31508001C205FFA384603210B2200F05AFA3846072194
S31508001C300B2200F055FA4FF4006330938DF8C66016
S31508001C408DF8C4408DF8C7608DF8C5404FF4C0576D
S31508001C50C4F20207384630A900F0F4F938460B21D9
S31508001C600A4600F03DFA322330938DF8C6608DF8A7
S31508001C70C4408DF8C7608DF8C5404FF40068C4F2BB
S31508001C800208404630A900F0DDF9404601210B2242
S31508001C9000F026FA404604210B2200F021FA4046BD
S31508001CA005210B2200F01CFA4FF4C04330938DF83F
S31508001CB0C6608DF8C4408DF8C7608DF8C5403846B3
S31508001CC030A900F0BFF938460D210B2200F008FABA
S31508001CD038460E210B2200F003FAFFF7CDFCFFF77A
S31508001CE01BFFFFF723FF0128FBD001A8FFF7D0FC55
S31508001CF00024019408944FF400730B930C944FF04E
S31508001D0000430F93202312931494159416944FF4BA
S31508001D10006309934FF4804306934FF0020A4FF08D
S31508001D2003094CF2F108C0F2070841F21967C0F23C
S31508001D302207A6B230465146FFF7FAFC60F31F4564
S31508001D4030464946FFF7F4FC60F30F05BD4218BF5D
S31508001D50454503D00134202CEBD109E0202C07D9C6
S31508001D6047F21860C0F600004FF4A17104F0D4FEE3
S31508001D7001A8A1B2FFF748FD38B947F21860C0F6C6
S31508001D80000040F2471104F0C7FE41F68063C2F234
S31508001D90000341F2D072C2F200029A60DB600022B0
S31508001DA01A605A604FF41041C4F202010B6141F205
S31508001DB08013C2F2000341F29010C2F2000098604C
S31508001DC01A60DB605A6040225A719A884FF4C860DC
S31508001DD060F30C029A808022DA70CB60FFF7E0FE8F
S31508001DE032B0BDE8F08700BF40F28C53C2F2000360
S31508001DF008221A7000225A7027229A706922DA700D
S31508001E005B221A7145225A71704700BF38B541F2F4
S31508001E108013C2F20003DB78DB091DD141F280147E
S31508001E20C2F200046588C5F30D0541F62070C2F2BA
S31508001E30000041F29011C2F200012A4605F030FB7B
S31508001E40E37843F08003E3704FF41043C4F20203CF
S31508001E5001229A60284638BD002038BD38B541F6BB
S31508001E608063C2F20003DB78DB0900D0FEE741F6A7
S31508001E709063C2F200031D8841F2D074C2F20004D6
S31508001E80204641F62071C2F200012A4605F008FBF9
S31508001E9041F68063C2F200039C6000221A6010219A
S31508001EA099705A60C5F30B059D80B022DA704FF41D
S31508001EB01043C4F2020301225A6038BD4FF470532E
S31508001EC0C4F202031B69002B0DDA4FF47053C4F2F7
S31508001ED0020340F22312C4F267525A6048F6AB1264
S31508001EE0CCF6EF525A6070474FF47053C4F20203AF
S31508001EF01A6942F000421A61704700BF4FF47053E6
S31508001F00C4F20203D86070474FF47053C4F2020358
S31508001F10DB6813F4803F1BD14FF47053C4F20203FD
S31508001F20DB6813F0100F15D14FF47053C4F2020397
S31508001F30DB6813F0EF0F0FD14FF47053C4F20203AE
S31508001F40D86800F0020000280CBF08200720704758
S31508001F5001207047052070470620704700B583B0FA
S31508001F6008238DF80730FFF7CFFF8DF807009DF897
S31508001F700730DBB2012B08D1FFF7C6FF8DF8070043
S31508001F809DF80730DBB2012BF6D09DF8070003B0A9
S31508001F905DF804FB70B50546002659B1012908BF4E
S31508001FA04FF4807606D0022914BF4FF440764FF4DA
S31508001FB00076FFE7FFF7D2FF082821D14FF47054C7
S31508001FC0C4F20204236923F44073236123691E4380
S31508001FD02661236923F0F8032361236943F002038A
S31508001FE01D432561236943F480332361FFF7B6FF58
S31508001FF0236923F002032361236923F0F80323618D
S3150800200070BD00BF70B505460E46FFF7A7FF082846
S3150800201016D14FF47054C4F20204236923F44073B2
S315080020202361236943F400732361236943F00103A1
S3150800203023612E60FFF792FF236923F001032361D2
S3150800204070BD00BFF0B400230125032605FA03F28C
S315080020500C681440944238D107685A0006FA02F40C
S31508002060E44327400760076891F804C00CFA02FCAD
S315080020704CEA070707600F79013FFFB2012F16D810
S3150800208087683C40846087684C7994403C43846008
S3150800209047689CB205FA04FC27EA0C0747604768BC
S315080020A091F806C00CFA04F4A4B23C434460C7682D
S315080020B09CB2640006FA04F427EA0404C460C468FF
S315080020C0CF7907FA02F22243C2600133102BBDD141
S315080020D0F0BC7047036919420CBF00200120704705
S315080020E010B401F007039B00C90800EB8100046ADD
S315080020F00F21994024EA01010162016A9A401143BD
S3150800210001625DF8044B704710B44FF46053C4F293
S3150800211002039B6803F00C03042B09D0082B0DD08F
S31508002120002B36D14FF41053C0F2F403036035E0A8
S315080021304FF4D853C0F2B70303602FE04FF460534F
S31508002140C4F202035C685A6802F03F0214F4800F76
S315080021504FF46053C4F202035B68C3F3881319BFD4
S315080021604FF4D854C0F2B7044FF41054C0F2F40434
S31508002170B4FBF2F101FB03F14FF46053C4F202031E
S315080021805A68C2F3014201325200B1FBF2F303600E
S3150800219004E04FF41053C0F2F40303604FF46052A6
S315080021A0C4F202029168C1F3031140F20803C2F2B5
S315080021B00003595CC9B2046824FA01F141609468C5
S315080021C0C4F382241C5DE4B221FA04F484609268A4
S315080021D0C2F342329B5CDBB2D940C1605DF8044B66
S315080021E0704700BF39B14FF46053C4F202031A6B4B
S315080021F01043186370474FF46053C4F202031A6B16
S3150800220022EA00001863704739B14FF46053C4F2EC
S3150800221002031A6C1043186470474FF46053C4F2F3
S3150800222002031A6C22EA00001864704739B14FF4A9
S315080022306053C4F202035A6C1043586470474FF453
S315080022406053C4F202035A6C22EA000058647047CD
S3150800225039B14FF46053C4F202031A691043186186
S3150800226070474FF46053C4F202031A6922EA000069
S315080022701861704739B14FF46053C4F202035A6AC1
S315080022801043586270474FF46053C4F202035A6A07
S3150800229022EA00005862704708B54FF40060012131
S315080022A0FFF7E8FF4FF400600021FFF7E3FF08BDE2
S315080022B010B44FF43053C4F201035C684168826875
S315080022C01143C26811430268114302690A4324F4A0
S315080022D0FD4424F07F042243017D0A435A605DF8D9
S315080022E0044B704748F2A003C4F2252318607047D0
S315080022F04FF43053C4F20103186070474FF430535B
S31508002300C4F20103186800F00300704710B40268AD
S315080023104FF43053C4F201039A60DC6824F4FF6476
S3150800232024F00704826841681143C2680A430069B9
S3150800233002432243DA605DF8044B70474FF430538A
S31508002340C4F201031869C0B2704700BF82B0002307
S31508002350019342F61443C4F2010303440193019B1B
S31508002360186802B0704700BF10B402684FF43053C3
S31508002370C4F201035A6242689A62DC6A24F0F704DE
S31508002380C2688168114302690A43406902432243CD
S31508002390DA625DF8044B70474FF43053C4F2010318
S315080023A0D3F88000704700BF4FF43053C4F20103DE
S315080023B0C3F88000704700BF4FF43053C4F20103DE
S315080023C05B6B18420CBF0020012070474FF4305356
S315080023D0C4F2010398637047DC23C4F2272318600C
S315080023E0704700BF30B585B004460D46038A23F40E
S315080023F040531B041B0CCA8813430382838923F4A6
S31508002400B05323F00C031B041B0C0989AA880A4342
S3150800241069890A4392B213438381838A23F44073FA
S315080024201B041B0CAA89134383826846FFF76CFEBC
S315080024304FF4A052C4F201024FF48053C4F20103D0
S315080024409C4218BF94420CBF039A029AA3891BB2F6
S31508002450002B02EB820202EB8202BDBF2B685B00F7
S31508002460B2FBF3F22968A4BF8900B2FBF1F248F285
S315080024701F53C5F2EB13A3FB02135B091D0164206E
S3150800248003FB1023A08900B200280BDADB003233E5
S3150800249048F21F51C5F2EB11A1FB0321C1F342110A
S315080024A029430AE01B01323348F21F51C5F2EB11EA
S315080024B0A1FB0321C1F34311294389B2218105B048
S315080024C030BD00BF29B183899BB243F40053838191
S315080024D07047838923F400531B041B0C83817047C0
S315080024E0C1F30801818070478088C0F308007047EF
S315080024F0038819420CBF00200120704782B04FF4B0
S315080025006053C4F202031A6842F001021A600022FC
S315080025109A60196821F0847121F48031196043F2B8
S315080025201001C2F200415960196821F4802119602E
S31508002530DA60009201921A6842F480321A604FF407
S315080025406052C4F20202136803F400330193009B3D
S3150800255001330093019B1BB9009BB3F5A06FF2D121
S315080025604FF46053C4F202031B6813F4003F14BF10
S31508002570012300230193019B012B46D14FF460539D
S31508002580C4F202031A6C42F080521A644FF4E04215
S31508002590C4F20002116841F4404111609A689A60D9
S315080025A09A6842F400429A609A6842F4A0529A6085
S315080025B045F20C42C0F240725A601A6842F08072C4
S315080025C01A604FF46052C4F20202136813F0007FD7
S315080025D0FBD04FF47053C4F2020340F205621A604E
S315080025E04FF46053C4F202039A6822F003029A6019
S315080025F09A6842F002029A604FF46052C4F20202EC
S31508002600936803F00C03082BFAD14FF46D43CEF20E
S3150800261000034FF000629A6002B0704732B1821828
S3150800262011F8013B00F8013B9042F9D1704700BF11
S31508002630CA7E8B7E43EA02230278032A01BF487DBD
S315080026400A7D42EA002243EA02431846704700BF61
S3150800265000F10B010023DA0142EA530310F8012BBB
S3150800266052FA83F3DBB28842F5D11846704700BFA9
S3150800267010B504460A46407804F134010123FEF7F2
S315080026805DFFD0BB94F8332294F8323243EA022233
S3150800269012B24AF65523CFF6FF739A422FD194F811
S315080026A06D2094F86C301B0443EA026294F86A3091
S315080026B0134394F86B2043EA022222F07F4244F245
S315080026C04613C0F254039A421BD094F8890094F832
S315080026D088301B0443EA006094F88630034394F874
S315080026E0870043EA002020F07F4044F24613C0F2F8
S315080026F05403C01A18BF012010BD032010BD0220C4
S3150800270010BD002010BD00BF2DE9F0410446037935
S315080027101BB3056B00F13407407839462A46012376
S31508002720FEF73EFFE0B900232371636A9D421AD380
S31508002730E26913449D4219D2E678012E19D94FF061
S315080027400108E2691544607839462A464346FEF789
S3150800275027FF013E012EF4D10EE00020BDE8F081EE
S315080027600120BDE8F0810020BDE8F0810020BDE829
S31508002770F0810020BDE8F0810020BDE8F08100BFAF
S3150800278038B504460D46036B8B420CD0FFF7BCFFE9
S3150800279058B9607804F134012A460123FEF7CEFEC3
S315080027A028B9256338BD002038BD012038BD012071
S315080027B038BD00BF08B588B103688BB1197889B1EF
S315080027C0D988828891420FD15878FEF79DFE00F08D
S315080027D00100002814BF0320002008BD092008BDF9
S315080027E0092008BD092008BD092008BD2DE9F041CA
S315080027F0154603681C78303C092C00F2B5815A78D6
S315080028003A2A40F0B1810233036000230B60002CA2
S3150800281040F0718140F27C53C2F200031C68002C20
S3150800282000F06C810C6023788BB16078FEF76CFE43
S3150800283010F0010F0BD1002D00F0638100F00400A9
S31508002840C0B2002814BF0A200020BDE8F08100208D
S3150800285020706070FEF73CFE10F0010F40F05481C6
S315080028601DB110F0040F40F0528120460021FFF7F9
S31508002870FFFE012818BF002517D194F8F631002B62
S3150800288000F0488194F8FD2194F8FC311B0443EAD2
S31508002890026294F8FA31134394F8FB5143EA05258A
S315080028A020462946FFF7E4FEFFE7032800F03581B6
S315080028B0002840F0358194F8402094F83F3043EAE8
S315080028C002231BB2B3F5007F40F02D8194F84B002C
S315080028D094F84A3053EA00200DD194F85B2094F816
S315080028E05A301B0443EA026294F85830134394F8AA
S315080028F0590043EA0020E06194F84410E1704B1E49
S31508002900DBB2012B00F2128194F84130A370002B40
S3150800291000F00F815A1E1A4240F00E8194F8466064
S3150800292094F8452042EA0622228112F00F0F40F061
S31508002930068194F8487094F8476056EA07260DD140
S3150800294094F8577094F85660360446EA076794F880
S3150800295054603E4394F8557046EA072694F843C0F7
S3150800296094F8427057EA0C2700F0EC8001FB00FC53
S3150800297007EB121161448E42C0F0E780761AB6FB67
S31508002980F3F3002B00F0E48040F6F576B3428CBFF3
S31508002990022601264FF6F578434500F2E880023311
S315080029A0A36125622F4467622944E162032E13D18D
S315080029B0002A40F0D08094F8631094F8622012043C
S315080029C042EA016194F860200A4394F8611042EAE9
S315080029D00122A2629B000EE0002A00F0BF80674435
S315080029E0A762022E0FBF5B0003225A4303F00103BE
S315080029F018BF03EB520303F2FF13B0EB532FC0F0DB
S31508002A00B0804FF0FF3323610023E360032E63D1C8
S31508002A10637194F8652094F8643043EA02222A44E4
S31508002A206261607804F134010123FEF787FD00280E
S31508002A3052D194F8332294F8323243EA022212B27F
S31508002A404AF65523CFF6FF739A4245D194F83720B4
S31508002A5094F836301B0443EA026294F83430134380
S31508002A6094F8352043EA022245F25223C4F2611350
S31508002A709A4231D194F81B2294F81A321B0443EA7D
S31508002A80026294F81832134394F8192243EA022290
S31508002A9047F27223C6F241139A421DD194F82322B3
S31508002AA094F822321B0443EA026294F82032134354
S31508002AB094F8212243EA0223E36094F81F2294F84B
S31508002AC01E321B0443EA026294F81C32134394F83C
S31508002AD01D2243EA02232361267040F27853C2F28C
S31508002AE000031A88013292B21A80E280002020631D
S31508002AF02071BDE8F0810B20BDE8F0810C20BDE80F
S31508002B00F0810020BDE8F0810320BDE8F0810A20AD
S31508002B10BDE8F0810D20BDE8F0810120BDE8F08117
S31508002B200D20BDE8F0810D20BDE8F0810D20BDE83F
S31508002B30F0810D20BDE8F0810D20BDE8F0810D2063
S31508002B40BDE8F0810D20BDE8F0810D20BDE8F081DB
S31508002B500D20BDE8F0810D20BDE8F0810D20BDE80F
S31508002B60F0810D20BDE8F08100230B6052E60233A8
S31508002B70A36125622F4467622944E162032617E7A9
S31508002B802DE9F0410D4601F109020369002B5ED0DB
S31508002B90416991F80C800B78202B1BD00E46002437
S31508002BA008F00807FFB203E016F8013F202B11D002
S31508002BB0052B08BFE52347B1A3F1410C5FFA8CFC4E
S31508002BC0BCF1190F9CBF2033DBB202F8013B01347C
S31508002BD0082CE9D10B7A202B22D0561C2E231370F1
S31508002BE00B7A202B1BD001F10804171D324608F07A
S31508002BF010085FFA88F603E014F8013F202B0FD07F
S31508002C0046B1A3F1410C5FFA8CFCBCF1190F9CBFCD
S31508002C102033DBB202F8013BBA42EDD100E032467E
S31508002C20CB7A2B72CC7F8B7F1B0443EA04630C7F21
S31508002C3023434C7F43EA04232B604C7E0B7E43EAF6
S31508002C400423AB80CC7D8B7D43EA0423EB800023F1
S31508002C501370AE6946B3EB6933B3036900240BB34B
S31508002C60028C4FF6FF739A4208BF00241AD0C76930
S31508002C70388890B10024A046414601F02BFC70B17B
S31508002C80EA69013AA2420CD90134321902F8010C58
S31508002C9037F8020F0028EFD104E0002402E00024F0
S31508002CA000E0002400233355BDE8F08110B5044642
S31508002CB0FFF72AFD0346002854D12378032B49D170
S31508002CC06379002B46D00023236304F1340104F50D
S31508002CD00D700B46002203F8012B8342FBD15523C6
S31508002CE084F83232AA2384F83332522384F83430F3
S31508002CF084F83530612384F83630412284F8372049
S31508002D00722084F8180284F8190284F81A2284F8C2
S31508002D101B32236984F81C32C3F3072284F81D2268
S31508002D201A0C84F81E221B0E84F81F32E36884F8F6
S31508002D302032C3F3072284F821221A0C84F82222AF
S31508002D401B0E84F82332607862690123FEF728FC9B
S31508002D5000236371607800210A46FEF757FC031CBE
S31508002D6018BF0123184610BD02398369023B9942F0
S31508002D703DBF8278C36A02FB01300020704700BF5E
S31508002D80F8B505460C4601295CD9836999425BD298
S31508002D900378022B28D0032B38D0012B56D101EB10
S31508002DA05106416A01EB5621FFF7EAFC002850D18B
S31508002DB0C6F308032B4493F834700136696A28462B
S31508002DC001EB5621FFF7DCFC002845D1C6F30806BF
S31508002DD0354495F8340047EA002014F0010F14BF73
S31508002DE00009C0F30B00F8BD416A01EB1421FFF797
S31508002DF0C7FCA0BB640004F4FF742B1993F83430A5
S31508002E002C4494F8350043EA0020F8BD416A01EBEA
S31508002E10D411FFF7B5FC28BBA40004F4FE742B19E3
S31508002E2093F8360093F83720120642EA004293F8E0
S31508002E30350042EA00202C4494F83430184320F038
S31508002E407040F8BD0120F8BD0120F8BD4FF0FF30F5
S31508002E50F8BD4FF0FF30F8BD4FF0FF30F8BD4FF02A
S31508002E60FF30F8BD4FF0FF30F8BD00BF70B504461F
S31508002E700D46E1808168012938D003689A69914234
S31508002E8036D271B91A78032A01D1996A49B900224A
S31508002E90E2601A89AA422DD99B6A03EB15132361AE
S31508002EA01BE09E783601B54210D32068FFF768FF0D
S31508002EB00146B0F1FF3F1FD001281FD923689B693F
S31508002EC098421DD2AD1BADB2AE42EED9E160206884
S31508002ED0FFF74AFF00EB1510206105F00F05236880
S31508002EE003EB451334336361002070BD022070BDC7
S31508002EF0022070BD022070BD012070BD022070BD89
S31508002F00022070BDF8B505460C461646012998BF3D
S31508002F1002237CD98369994228BF022377D2037892
S31508002F20022B40D0032B50D0012B18BF02236BD1A4
S31508002F3001EB5107416A01EB5721FFF721FC0346D4
S31508002F40002861D1C7F3080314F001041FBFEA186B
S31508002F5092F8342002F00F02F1B21ABF42EA0112C7
S31508002F60D2B2F2B22B4483F83420013701232B71F5
S31508002F70696A284601EB5721FFF702FC0346002839
S31508002F8042D1C7F3080714B1C6F3071607E0EA19D2
S31508002F9092F8342022F00F02C6F3032616432F4474
S31508002FA087F8346030E0416A01EB1421FFF7E8FB4B
S31508002FB0034648BB640004F4FF742A1982F8346097
S31508002FC0C6F3072682F835601EE0416A01EBD41184
S31508002FD0FFF7D6FB0346B8B9A40004F4FE742A1911
S31508002FE092F8371009062C4401F070410E4384F814
S31508002FF03460C6F3072182F83510310C82F8361092
S31508003000360E82F83760FFE701222A71FFE7184675
S31508003010F8BD00BF2DE9F0410546884631B9C668B6
S3150800302076B183699E4228BF01260AE0FFF7A8FE0B
S31508003030012847D9AB69984228BF464601D24DE0D8
S315080030400126344602270134AB699C4202D3012E7D
S315080030503BD93C4628462146FFF792FE38B1B0F1E7
S31508003060FF3F18BF012833D0B442ECD132E02646E0
S31508003070284621466FF07042FFF744FF0346D0F119
S31508003080010038BF0020B8F1000F08BF002028B1A2
S31508003090284641462246FFF735FF03465BB9EE60F0
S315080030A02B69B3F1FF3F18D0013B2B6101236B71EC
S315080030B02046BDE8F081012B14BF01204FF0FF30F8
S315080030C0BDE8F0810120BDE8F0810020BDE8F0816F
S315080030D0BDE8F0810020BDE8F0812046BDE8F0811A
S315080030E02DE9F84304460E46C5880135ADB2002DD4
S315080030F06AD00369002B6AD015F00F075BD101333C
S315080031000361C16821B903681B89AB4262D952E0E1
S3150800311000688378013B13EA15134CD1FFF730FE9C
S315080031208046012859D9B0F1FF3F59D020688369F4
S31508003130984539D3002E56D0E168FFF76BFF8046D5
S31508003140002853D0012854D0B0F1FF3F54D020684E
S31508003150FFF7DAFA002852D1236803F13401002375
S315080031601A46CA540133B3F5007FFAD126683046A9
S315080031704146FFF7F9FD306300264FF001090CE0E0
S3150800318083F804902068FFF7BFFA00283AD123682D
S315080031901A6B01321A630136F6B223689A78B2427C
S315080031A0EED81A6B921B1A63C4F80C802068414645
S315080031B0FFF7DAFD2061E580236803EB4713343314
S315080031C063610020BDE8F8830420BDE8F883042085
S315080031D0BDE8F8830420BDE8F8830220BDE8F8833B
S315080031E00120BDE8F8830420BDE8F8830720BDE880
S315080031F0F8830220BDE8F8830120BDE8F8830120A2
S31508003200BDE8F8830120BDE8F88300BF2DE9F04F3B
S3150800321089B005460021FFF729FE002840F0AC805A
S315080032204FF0FF09C8464F4647F2C061C0F6000195
S31508003230029101F10C0204924FF6FF7A4FF0000B4F
S3150800324028682969FFF79CFA002840F096806C697F
S315080032502678002E00F09280E37A03F03F02E52EEE
S315080032607FD013F0080F04D00F2A18BFB8467BD1B9
S3150800327001E00F2A58D1EB690193002B74D016F0A0
S31508003280400F06D094F80D9006F0BF06EB882B8405
S3150800329003E0B04518BFB84666D1617B039149453E
S315080032A018BFB84660D1237823F04003013B03EBEF
S315080032B0430203EB82020592029A02F1FF394FF0AC
S315080032C001080796059E06954546DDF8108019F80B
S315080032D0013FE2185078E35C43EA00207DB101F033
S315080032E01FF90546FE2E56D8731C0593019931F829
S315080032F0160001F015F985424FD1059E01E05045AB
S315080033004DD1C145E3D1A8460596079E069D23786B
S3150800331013F0400F39D0B8F1000F36D0059A01994D
S3150800332031F812308BB33BE0B8F1000F04D12046D8
S31508003330FFF78EF9484523D0A5F820A0AB69DA7ABD
S3150800334012F0010F08BF04F10B0002D00BE0844213
S3150800335018D014F8011B13F8012B9142F7D0B84680
S3150800336002E0B84600E0B84628465946FFF7B8FED8
S3150800337000283FF465AF07E016E015E0042013E0E7
S31508003380002011E000200FE00EE0013E5FFA86F80B
S31508003390DDF80C90E8E7069D02E0069D00E0069D34
S315080033A0DDF80C90B846DFE709B0BDE8F08F00BF3E
S315080033B02DE9F04F87B0814688460B782F2B18BF2A
S315080033C05C2B08BF01F101080023836098F80030E0
S315080033D01F2B07D80021FFF749FD03460022C9F82D
S315080033E014207AE14FF0010A47F22C6BC0F6000B65
S315080033F047F23861C0F60001049147F24062C0F610
S315080034000002059298F800302F2B18BF5C2B08D1C4
S3150800341008F10103984613F8012B2F2A18BF5C2AD6
S31508003420F8D0D9F81C5098F800002F2818BF1F2884
S315080034302CD95C2800F02D81AF1E4646544607E07D
S315080034405C2B00F02881B2F5807F00F0418114469C
S31508003450514601F03FF80146002800F039817F28DF
S3150800346009D8222900F034815A4612F8013F13B1CF
S315080034709842FAD12CE127F8021F621C16F8013F80
S3150800348018462F2B18BF1F2BDAD801E00024524606
S3150800349090441F2898BF042601D90026FFE7002C70
S315080034A000F0168104F10043013B5A0035F8133049
S315080034B02E2B18BF202B40F0F080931C2B4407E0DE
S315080034C033F8042C023B2E2A18BF202A40F0E58048
S315080034D0013CF5D1FCE003F8011B8342FBD12B88A4
S315080034E0202B18BF2E2B40F0E480284600230133FA
S315080034F030F8021F202918BF2E29F8D0002B00F01B
S31508003500D98046F00306D5E0013C05D10821039190
S3150800351000220192029205E0023A32F8021C2E2994
S31508003520F2D1F3E75F1C35F81300002861D0202894
S3150800353008D0E31B18BF01232E2814BF002203F06E
S3150800354001021AB146F003063B46EBE7019A0399D6
S31508003550BC4218BF8A4214D30B2903D146F003068E
S31508003560029A49E00BB146F00306A74243D8029AED
S315080035709300DBB2029323460B21039108220192A2
S31508003580D0E77F280DD9002100F0A4FF03460028C4
S3150800359000F0A08005990B4413F8800C46F002064B
S315080035A050B101462B2807D0049A12F8013F002B88
S315080035B000F087809942F8D146F003065F2010E0B4
S315080035C0029A42F0020202920BE0A0F161039BB25A
S315080035D0192B9FBF029B43F001030293203898BF23
S315080035E080B2D9F81830019958543B4601310191F7
S315080035F098E7029A00E0029AD9F818301978E5296E
S3150800360004BF05211970039B082B02BF9200D2B292
S315080036100292029901F00C030C2B03D001F003026D
S31508003620032A01D146F0020616F0020F0AD10299C2
S3150800363001F00302012A08BF46F01006042B08BF52
S3150800364046F00806D9F81830DE724846FFF7DEFD60
S31508003650D9F81830DA7A034648B104283DD102F081
S315080036600403DBB2002B14BF0346052335E012F032
S31508003670040F32D1D9F81410CB7A13F0100F06D0F4
S31508003680D9F80000FEF7D4FFC9F80800BAE6052302
S3150800369023E0002452469044FFE66700EA194FF0FB
S315080036A0000325F81430D9F8183003F10B0020214F
S315080036B011E700232F4437F8021C2E293FF426AFC2
S315080036C022E7A0F141039BB2192B7FF679AF7CE77D
S315080036D0062302E046F002066EE7184607B0BDE884
S315080036E0F08F00BF2DE9F04F83B0044689464FF0AE
S315080036F0FF0B5E460425D84647F2C06AC0F6000AA4
S315080037000AF10C030093002770E02068FFF738F8E9
S31508003710054600286ED162691378002B74D0D17AD9
S31508003720E52B18BF2E2B59D001F03F01082914BFED
S3150800373000200120484518BF464651D10F2943D1DC
S3150800374013F0400F06D092F80DB003F0BF03E188DE
S31508003750218403E09E4218BF464641D192F80DE007
S31508003760DE4518BF46463BD1D4F81CC0117801F097
S315080037703F01013901EB410501EB85050AF1FF31EE
S3150800378001260193DDF800B011F8013FD018407802
S31508003790D35C43EA002036B1FE2D32D82CF815004A
S315080037A00646013503E04FF6FF73984229D159457D
S315080037B0EAD1019B127812F0400F1ED0FE2D98BF59
S315080037C02CF8157019D91CE010461EB9FEF740FFF3
S315080037D058451BD04FF6FF73238417E04646FFE78C
S315080037E020463946FFF77CFC054618B921690029A9
S315080037F08BD15DB10023236108E0013BDEB2F346BD
S31508003800EEE7F3464646EBE70425F3E7284603B01A
S31508003810BDE8F08F2DE9F0410446C588018C4FF6C6
S31508003820FF73994208BF2946FFF720FB0346D0B924
S31508003830E52701264FF0000820682169FEF7A0FF5A
S31508003840034668B96269177022681671E288AA4247
S3150800385009D220464146FFF743FC03460028EBD031
S31508003860042B08BF02231846BDE8F0812DE9F04174
S3150800387004460E46012998BF02212BD983699E4228
S3150800388028BF022126D200274FF0010820463146DC
S31508003890FFF776FA0546C0B1012818D0B0F1FF3F08
S315080038A017D0204631463A46FFF72CFB014688B921
S315080038B02369B3F1FF3F1EBF0133236184F80580F6
S315080038C0A369AB4206D92E46E0E7002102E00221B1
S315080038D000E001210846BDE8F08100BF70B582B05E
S315080038E0054616461C460B22FEF798FE052C0BD9F4
S315080038F0B21EE30343EA540432F8023F13FA84F48F
S31508003900A4B25388002BF4D1072204F00F0101F169
S315080039103003392B88BF01F13703013A00A9114456
S315080039204B702409F1D114467E2102AB134403F8E7
S31508003930081C62B12B78202B0BD0294600230133B3
S31508003940A34207D011F8010F2028F8D102E000237E
S3150800395000E000232020072A9FBF02A9891811F832
S31508003960081C013288BF0146E9540133072BF2D9F6
S3150800397002B070BD2DE9F04F87B004468769C66965
S3150800398003A839460C22FEF749FE9DF8173013F0B6
S31508003990010F21D00023FB72E3610125384603A9F4
S315080039A032462B46FFF79AFF2046FFF72FFC0346C1
S315080039B020B90135ADB2642DF0D1D5E0642D08BF2C
S315080039C0072000F0EF80042B18BF184640F0EA8065
S315080039D09DF81730FB72E6619DF8173013F0020F59
S315080039E008BF012716D033883BB1002301339BB2A9
S315080039F036F81320002AF9D100E0002319334EF6D1
S31508003A004F42C4F6C46282FB0317DB17C3EBA70752
S31508003A10BFB2FFE720460021FFF728FA0346002831
S31508003A2040F0BF800025A846012620682169FEF7D8
S31508003A30A7FE0346002840F0B48063691B78E52B8F
S31508003A4018BF002B03D10135AF4201D18EE04546A0
S31508003A5020463146FFF744FB03460028E5D0A0E0A0
S31508003A60E188C9EB0101204689B2FFF7FFF9034651
S31508003A70002840F09680A069FEF7EAFD01904FF015
S31508003A8000084FF6FF7547F2C066C0F60006FF2726
S31508003A9020682169FEF774FE0346002840F08180FD
S31508003AA0D4F81CA061695FFA89FB019A4A734FF042
S31508003AB00F03CB7281F80C8081F81A8081F81B807D
S31508003AC00BF1FF3303EB430003EB8000012243466F
S31508003AD002E070462B460132AB424ED000F1010E91
S31508003AE03AF81030B01810F8010C0B5408444FEA95
S31508003AF0132C80F801C0002B49D070460C2AEAD94D
S31508003B00AB4202D03AF810300BB94BF0400B81F8B3
S31508003B1000B023684FF00101197120464146FFF7AE
S31508003B20DFFA034600283CD109F1FF391FFA89F963
S31508003B30B9F1000FACD12DE0636903F12001002231
S31508003B4003F8012B8B42FBD16069A1690B22FEF7B2
S31508003B5065FD6369A269D27A02F018021A732368AE
S31508003B6001221A7100201DE007201BE0013F1FFA01
S31508003B7087F9B9F1000F0DD072E706EB020E1EF8B1
S31508003B8001EC01F80E708E448EF80170B6E70C2A27
S31508003B909FD9BAE720682169FEF7F2FD0028CBD045
S31508003BA000E0184607B0BDE8F08F00BF88B940F2BC
S31508003BB07C53C2F200031B680BB100221A7009B1CC
S31508003BC000230B7040F27C53C2F2000319600020F8
S31508003BD070470B20704700BF2DE9F0438FB0019165
S31508003BE015460446002800F094800023036001A8C7
S31508003BF005A902F01E02FEF7F9FD002840F08B80A9
S31508003C0005F01F0702AB0B9340F27833C2F20003AC
S31508003C100C9305A80199FFF7CBFB0A9E03460028DB
S31508003C207FD1002E78D17BE05BB1042B40F08580F4
S31508003C3005A8FFF79FFE47F008070A9E034638B116
S31508003C407BE0F37A13F0110F70D115F0040F6FD1E2
S31508003C5017F0080F3CD0FDF70BFDB073C0F3072330
S31508003C60F373030C3374000E70740025F572357700
S31508003C707577B577F577DDF8148040463146FEF757
S31508003C80D7FCB576F57635757575012388F8043051
S31508003C900546E8B1D8F8309040462946FFF7E6FDD4
S31508003CA00346002849D10598013DC5604946FEF7F7
S31508003CB067FD03460AE0F37A13F0100F3AD115F0C0
S31508003CC0020F05D013F0010F36D101E0002B34D1D5
S31508003CD017F0080F18BF47F02007059D2B6BE36107
S31508003CE02662A77128463146FEF7A2FC2061F27FBC
S31508003CF0B37F1B0443EA0263327F1343727F43EAAE
S31508003D000223E3600020A060A0612560EB88A38001
S31508003D1014E0092012E011E015F01C0F91D1CAE752
S31508003D20062315F01C0F7FF47FAFCFE7072304E0C7
S31508003D30082302E0042300E0072318460FB0BDE875
S31508003D40F08300BF2DE9F04F83B004460F46904636
S31508003D501E4600233360FEF72DFD002840F0BF8085
S31508003D60A37913F0800F18BF022040F0BC8013F02F
S31508003D70010F08BF072000F0B680E568A368ED1AB2
S31508003D80A84538BF4546002D00F0AA8004F1240353
S31508003D900193A368C3F30802002A40F086802068CE
S31508003DA090F802A00AF1FF3A0AEA532A1AF0FF0A23
S31508003DB017D10BB9206902E06169FEF7E1FF012816
S31508003DC005D8A37963F07F03A37102208BE0B0F1D5
S31508003DD0FF3F05D1A37963F07F03A371012082E039
S31508003DE06061D4F8008040466169FEF7BDFF8146F0
S31508003DF028B9A37963F07F03A371022073E0D14445
S31508003E005FEA552B29D098F802300BEB0A029A4242
S31508003E1088BFCAEB030B98F8010039464A465FFA91
S31508003E208BF3FDF78BFB28B1A37963F07F03A371AE
S31508003E30012058E0A37913F0400F0BD0A369C9EB12
S31508003E400300834506D907EB402001994FF4007219
S31508003E50FEF7E4FB4FEA4B2B35E0A2694A4522D030
S31508003E60A37913F0400F10D098F8010001990123A7
S31508003E70FDF796FB28B1A37963F07F03A3710120B0
S31508003E8031E0A37923F04003A37123685878019998
S31508003E904A460123FDF752FB28B1A37963F07F0355
S31508003EA0A37101201FE0C4F81890A168C1F30801A6
S31508003EB0C1F5007B5D4538BFAB4621443846243101
S31508003EC05A46FEF7ABFB5F44A3685B44A3603368BE
S31508003ED05B443360B5EB0B057FF45BAF02E002E0B1
S31508003EE0002000E0002003B0BDE8F08F2DE9F04F78
S31508003EF083B004460F4615461E4600233360FEF778
S31508003F0059FC002840F0DA80A37913F0800F18BF17
S31508003F10022040F0D48013F0020F08BF072000F0FB
S31508003F20CE80E368DD4280F0BE80002D00F0BB80C5
S31508003F3004F124030193A368C3F30802002A40F09E
S31508003F409580206890F802B00BF1FF3B0BEA532BE3
S31508003F501BF0FF0B21D13BB9236963B90021FFF799
S31508003F6059F80346206103E06169FFF753F80346F1
S31508003F70002B00F09880012B05D1A37963F07F030D
S31508003F80A37102209BE0B3F1FF3F05D1A37963F04B
S31508003F907F03A371012092E06361A37913F0400FB8
S31508003FA011D0236858780199A2690123FDF7F8FA18
S31508003FB028B1A37963F07F03A37101207FE0A37979
S31508003FC023F04003A371D4F8008040466169FEF7E8
S31508003FD0CBFE814628B9A37963F07F03A37102203B
S31508003FE06DE0D9445FEA552A29D098F802300AEBE1
S31508003FF00B029A4288BFCBEB030A98F801003946B0
S315080040004A465FFA8AF3FDF7CBFA28B1A37963F03B
S315080040107F03A371012052E0A369C9EB03018A4516
S315080040200AD9019807EB41214FF40072FEF7F6FA18
S31508004030A37923F04003A3714FEA4A2A28E0A3692B
S315080040404B4511D0A268E3689A420DD298F8010050
S3150800405001994A460123FDF771FA28B1A37963F05D
S315080040607F03A37101202AE0C4F81890A068C0F362
S315080040700800C0F5007A554538BFAA4620442430C2
S3150800408039465246FEF7CAFAA37943F04003A371AC
S315080040905744A3685344A360336853443360B5EB6D
S315080040A00A057FF448AFA368E268934288BFE360D5
S315080040B0A37943F02003A371002000E0FFE703B0D3
S315080040C0BDE8F08F38B50446FEF774FB002849D1E1
S315080040D0A37913F0200F46D013F0400F0DD02146D8
S315080040E051F8243B5878A2690123FDF759FA0028AC
S315080040F03BD1A37923F04003A3712068E169FEF759
S315080041003FFB002833D1256AEB7A43F02003EB7294
S31508004110E3682B77A3891B0A6B77E389AB77E37B85
S31508004120EB772369AB76C3F30722EA761B0C2B756C
S315080041301B0A6B75FDF79CFAA875C0F30723EB7588
S31508004140030C2B76000E68760023AB74EB74A37908
S3150800415023F02003A371236801221A712068FEF751
S31508004160A5FD38BD38BD002038BD012038BD38BD95
S3150800417010B50446FFF7A6FF034608B900222260D9
S31508004180184610BD70B504460D46FEF713FB002809
S3150800419040F0BD80A37913F0800F40F0B980E26843
S315080041A0AA4205D203F00203DBB2002B08BF15466C
S315080041B0A2680023A360002D00F0AC8020688678F2
S315080041C076026AB1013A691EB1FBF6F1B2FBF6F363
S315080041D0994205D373421A40A260AD1A616918E084
S315080041E02169A9B9FEF716FF0146012805D1A37969
S315080041F063F07F03A371022070BDB0F1FF3F18BFC3
S31508004200206105D1A37963F07F03A371012070BDF6
S315080042106161002940D0B5422BD9A27912F0020F6C
S3150800422005D02068FEF7F6FE014620B920E0206892
S31508004230FEF7A6FD0146B1F1FF3F05D1A37963F06C
S315080042407F03A371012070BD012903D922689269F1
S31508004250914205D3A37963F07F03A371022070BD51
S315080042606161A2683244A260AD1BAE42D5D300E0BC
S315080042703546A2682A44A260C5F3080272B12068CE
S31508004280FEF772FD28B9A37963F07F03A3710220B4
S3150800429070BD00EB552502E0002500E00025A36867
S315080042A0C3F3080343B3A269AA4225D0A37913F03E
S315080042B0400F11D0214651F8243B58780123FDF7C9
S315080042C06FF928B1A37963F07F03A371012070BD4C
S315080042D0A37923F04003A371214651F8243B58786B
S315080042E02A460123FDF72AF928B1A37963F07F034B
S315080042F0A371012070BDA561A368E26893420BD93A
S31508004300E360A37943F02003A371002070BD70BD5C
S31508004310022070BD002070BD002070BD30B58FB082
S315080043200EAB43F8340D0D46184605A90022FEF7D4
S315080043305DFA0446A0B902AB0B9340F27833C2F299
S3150800434000030C9305A80199FFF732F8044638B91B
S315080043500A9B23B105A82946FEF712FC00E00624AD
S3150800436020460FB030BD00BF30B599B018AB43F842
S315080043705C0D18460FA90122FEF738FA03460028F5
S315080043804DD103AB159340F27833C2F2000316936E
S315080043900FA80199FFF70CF8034600283FD1149996
S315080043A0062300293BD0CC7A14F0010F18BF072347
S315080043B035D124E0012D98BF022330D906A80FA9CC
S315080043C02422FEF72BF9089506A80221FEF74EFDD2
S315080043D0034620BB06A80021FFF784F90346E8B187
S315080043E0042814D01BE02DB10F982946FFF73EFA92
S315080043F00346A0B90F98FEF759FC03460FE00F983D
S31508004400FEF716F9054614F0100FD3D1FFE70FA8EB
S31508004410FFF700FA03460028E5D000E00723184610
S3150800442019B030BD2DE9F04383B081469046054664
S3150800443000244E1E012711E0404601A93A466B4664
S31508004440FFF780FC009B012B0AD19DF804300D2B49
S3150800445004D005F8013B01340A2B01D0A642EBDC57
S3150800446000232B709C4214BF4846184603B0BDE88B
S31508004470F08300BF30B583B004460D460A2802D142
S315080044800D20FFF7F7FF02A901F8084D28466946EF
S31508004490012201ABFFF72AFD0198012814BF4FF04E
S315080044A0FF30012003B030BD70B505460E460078D2
S315080044B060B100243146FFF7DDFFB0F1FF3F08D0B9
S315080044C0013415F8010F0028F4D101E0002070BD71
S315080044D0204670BD7F2821D941B9C7281EBF47F697
S315080044E0B002C0F6000201230AD112E0FF2814D850
S315080044F0803847F6B003C0F6000333F8100070475B
S3150800450032F8021F814205D001339BB2802BF7D1C6
S3150800451000E000238033D8B270470020704700BF00
S3150800452061280CD047F2D062C0F6000200210131A2
S3150800453032F8023F53B18342F9D10BB970470021D3
S3150800454047F6B013C0F6000333F81100704700BFF2
S3150800455030B4013A8D18A94214D20B461C785A7801
S3150800456002EB042292B2104480B2824284BF013028
S3150800457080B202339D42F1D8CB432B4423F001038A
S3150800458002331944A94207D10B781B02184480B29A
S31508004590834284BF013080B230BC704738B541F6DB
S315080045A02074C2F20004657C143D237C05EB0325C8
S315080045B0ADB2284480B204F11A010822FFF7C8FFF9
S315080045C004F122012A46FFF7C3FF034620B1000A79
S315080045D040EA032080B238BD4FF6FF7038BD00BFF1
S315080045E070B4C4780C44E4B241F69863C2F200038E
S315080045F0DC700D0A82782A44D2B29A7046785E70C8
S315080046000078187095420DD90136F6B241F69863CE
S31508004610C2F200035E702EB941F69863C2F2000337
S3150800462001301870C9B28C4217DA0132D2B241F69B
S315080046309863C2F200039A707AB941F69863C2F297
S3150800464000035A780132D2B25A7032B941F69863E9
S31508004650C2F200031A7801321A7070BC704700BFA4
S3150800466010B5014641F6A464C2F200042068083079
S31508004670FFF7B6FF226841F69863C2F2000319787D
S3150800468011725978517299789172DB78D37210BD8C
S3150800469008B5002006491422FFF75AFF034620B141
S315080046A0000A40EA032080B208BD4FF6FF7008BD35
S315080046B02E1F002008B50620FFF770FF08BD00BFB3
S315080046C041F61073C2F2000300221A8041F6A8636D
S315080046D0C2F200035A7640F29453C2F20003012252
S315080046E01A7040F28853C2F200034FF480621A80AF
S315080046F0704700BF40F29453C2F2000300221A70BA
S3150800470041F61073C2F200031B882BB941F61073E9
S31508004710C2F200031880704740F29453C2F20003B5
S3150800472001221A70704700BF38B541F6A463C2F279
S3150800473000031C6841F6A063C2F20003A54A1A608A
S3150800474041F69463C2F200031A60032813D1637E0C
S3150800475003F00F03032B40F05B87238A002B40F0FE
S31508004760578741F69C63C2F2000308221A7001F0CB
S3150800477071FB00F097BD022840F09E8040F28453FA
S31508004780C2F20003DA780132D2B2DA70C2B940F264
S315080047908453C2F200039A780132D2B29A707AB977
S315080047A040F28453C2F200035A780132D2B25A70E8
S315080047B032B940F28453C2F200031A7801321A70F1
S315080047C041F69063C2F2000300221A8042F2625355
S315080047D0C2F200031A80637E03F0FD02052A09D19E
S315080047E0A37E0133DBB2A376782B04BF002363765E
S315080047F000F00EBF002B00F00B87228A002A4CD04F
S31508004800A27E511EA176002A40F00287E27E082A7F
S3150800481005D0591EC9B2012914D8052A12D1002378
S31508004820637641F69C63C2F2000380221A7001F097
S3150800483011FB41F62073C2F20003142283F82F20DD
S3150800484000F063BE042A9DBF03219140C9B23021FE
S31508004850A1760132E27603F00F03013B072B00F243
S31508004860D786DFE813F05D0208001000AC04D50611
S31508004870AC04D506AC0441F62073C2F2000300224C
S3150800488083F82F2053E241F69C63C2F20003042208
S315080048901A7001F0DFFA00F056BD03F00F03032B80
S315080048A040F0B68641F69C63C2F2000308221A70ED
S315080048B001F0D0FA00F0F6BC41F62073C2F200030C
S315080048C09B7B452B40F0A48641F62073C2F2000379
S315080048D0197C5A7C02EB012041F69063C2F2000370
S315080048E01B88984200F3948684B241F69063C2F21C
S315080048F000031C8041F62073C2F200031B7D13F0EF
S315080049003F0F40F0858641F62073C2F200035B7DB7
S31508004910002B40F07D8641F61C73C2F200031D8809
S315080049202DB941F61C73C2F200035B88A3B141F6A8
S315080049302073C2F20003DB8BAB4240F0698641F676
S315080049402072C2F2000241F61C73C2F20003128CF6
S315080049505B889A4240F05C86FFF79AFE4FF6FF7333
S31508004960984240F0558641F62073C2F20003DB7D7B
S31508004970062B31D0012B40F04B8641F62073C2F24C
S31508004980000393F82230082B40F0428641F6207344
S31508004990C2F20003002283F822209A8C4FF6F6739F
S315080049A09A4241F62073C2F200038CBF09320832DC
S315080049B09A8441F62073C2F200035A8BDA839A8BE3
S315080049C01A845D8341F61C72C2F2000252889A83E9
S315080049D000F017BE561F0020FFF76CFE4FF6FF7358
S315080049E0984240F0158641F6A863C2F20003597E44
S315080049F081B341F62072C2F2000241F6A863C2F200
S31508004A000003928C9B889A4224D141F62072C2F206
S31508004A10000241F6A863C2F20003528CDB889A4270
S31508004A2018D141F62072C2F2000241F6A863C2F21A
S31508004A300003528B1B889A420CD141F62072C2F2AF
S31508004A40000241F6A863C2F20003928B5B889A4281
S31508004A5000F08D8141F62073C2F2000393F82F30DF
S31508004A6003F03F03022B1CD141F62073C2F2000368
S31508004A709A8C40F28053C2F200031A8040F2945393
S31508004A80C2F200030021197041F61073C2F2000346
S31508004A901B8893427BD040F29453C2F20003012252
S31508004AA01A7041F62073C2F2000393F82F3013F000
S31508004AB0040F40F0AD8541F62073C2F200031422BC
S31508004AC083F82F2041F69062C2F200022821118055
S31508004AD0502283F82E2093F8295093F82D2083F836
S31508004AE0292093F8284093F82C2083F8282083F867
S31508004AF02C4093F8270093F82B2083F8272083F877
S31508004B002B0093F8262040F29451C2F200010A7055
S31508004B1093F82A1083F8261083F82A20691CC9B24C
S31508004B2083F82D10C1B9611CC9B241F62073C2F2CF
S31508004B30000383F82C1079B9411CC9B241F62073D9
S31508004B40C2F2000383F82B1031B941F62073C2F282
S31508004B500003013283F82A2041F62073C2F20003CB
S31508004B60598C40F28052C2F2000211809A8C5A8403
S31508004B7099845A8BDA839A8B1A8441F61C72C2F28C
S31508004B8000021188598352889A8300F00DBD41F6B8
S31508004B90A863C2F200035B7E23B1072B40F04C8565
S31508004BA000F042BD41F6A461C2F2000141F6A863D5
S31508004BB0C2F200030B6003219976197600219975D4
S31508004BC00420D875D9769A8041F62074C2F200047A
S31508004BD0628CDA80628B1A80A28B5A800120587602
S31508004BE040F28452C2F2000211781973517859734F
S31508004BF091789973D278DA73188294F82920DA7240
S31508004C0094F828209A7294F827205A7294F8262045
S31508004C101A72FFF725FD94F82E3003F0F002502A99
S31508004C207ADD1B095C1FA40040F29553C2F200030B
S31508004C301A78002341F62071C2F200015AE0CA1818
S31508004C4092F8362072B940F29451C2F200010B7004
S31508004C5040F29553C2F200031A7041F6A864C2F2F4
S31508004C6000045DE0012A02D10133DBB242E0022AE8
S31508004C702BD10D1895F83750042D26D140F29452B1
S31508004C80C2F20002137040F29553C2F200030222E8
S31508004C901A7041F62073C2F20003034493F83820D1
S31508004CA093F8393043EA022240F28053C2F20003F5
S31508004CB01A8040F20A639A4238BF134641F6A8643E
S31508004CC0C2F200046382A3822AE0084490F83700FF
S31508004CD070B940F29451C2F200010B7040F295533C
S31508004CE0C2F200031A7041F6A864C2F2000417E083
S31508004CF00344DBB21846A342A1DB40F29451C2F248
S31508004D0000010B7040F29553C2F200031A7041F687
S31508004D10A864C2F2000403E041F6A864C2F20004E3
S31508004D2041F62073C2F20003102283F82F2041F6C1
S31508004D302073C2F2000393F82F2042F0020283F890
S31508004D402F20022283F83620042283F837200622F1
S31508004D5083F838200A2283F8392041F69062C2F295
S31508004D6000022C211180602283F82E20DAE341F616
S31508004D70A463C2F2000341F6A862C2F200021A60F6
S31508004D8041F69C63C2F2000300221A7041F62073B2
S31508004D90C2F2000393F82F3013F0040F0ED041F639
S31508004DA0A863C2F200035A7641F69C63C2F2000376
S31508004DB020221A7001F04EF800F02ABC41F6207243
S31508004DC0C2F2000292F82E000009800040F29452C6
S31508004DD0C2F200021070143C201A80B241F69062AA
S31508004DE0C2F20002108001F00F01022903D103F07C
S31508004DF03F02122A1DD010B913F0030F19D041F63D
S31508004E002071C2F2000141F6A862C2F20002C98C02
S31508004E101289914240F06E8341F62071C2F2000178
S31508004E2041F6A862C2F20002098D5289914240F009
S31508004E30618313F0100F77D041F6A863C2F200031E
S31508004E40198A002970D003F10C00FFF7C9FB41F657
S31508004E502073C2F2000393F82A4041F69863C2F21F
S31508004E6000031B78A3425FD141F62073C2F2000308
S31508004E7093F82B0041F69863C2F200035B788342ED
S31508004E8052D141F62073C2F2000393F82C1041F672
S31508004E909863C2F200039B788B4245D141F6207392
S31508004EA0C2F2000393F82D2041F69863C2F200037C
S31508004EB0DB78934238D141F6A863C2F200031C732B
S31508004EC058739973DA73DB7E03BB41F6A863C2F2A3
S31508004ED00003987D197E9A7E891AA1EBD001C9B282
S31508004EE0CAB20844C0B2987512F0800F1CBF4A4275
S31508004EF0D2B241F6A863C2F20003D97DA1EB9101B3
S31508004F000A44D2B2DA7502EBD0021A7641F69C63ED
S31508004F10C2F2000301221A7041F6A863C2F2000326
S31508004F201A7E9A7600221A8241F6A863C2F2000314
S31508004F305A7E02F00F03013B072B00F26983DFE874
S31508004F4013F008003A00040151029B02C702D90275
S31508004F50390241F69C63C2F200031B7813F0010F75
S31508004F6000F0568341F6A863C2F2000303225A767C
S31508004F7041F69C62C2F200024021117000221A8298
S31508004F8041F69063C2F20003188838B141F69C6373
S31508004F90C2F2000342221A70FFF762FB42F2625322
S31508004FA0C2F2000300221A8000F054FF41F6A864FA
S31508004FB0C2F2000476E141F69C63C2F200031B7854
S31508004FC013F0010F00F0B18041F62073C2F200031E
S31508004FD093F82F3003F03F03122B40F0A68041F6DA
S31508004FE02073C2F2000393F82E3003F0F002502A21
S31508004FF06DDD1B095C1FA40040F29553C2F2000345
S315080050001A78002341F62071C2F2000152E0CA184C
S3150800501092F8362052B940F29451C2F200010B7050
S3150800502040F29553C2F200031A7050E0012A02D1E9
S315080050300133DBB23EE0022A2BD10D1895F8375022
S31508005040042D26D140F29452C2F20002137040F2A7
S315080050509553C2F2000302221A7041F62073C2F277
S315080050600003034493F8382093F8393043EA0222C0
S3150800507040F28053C2F200031A8040F20A639A4251
S3150800508028BF1A4641F6A863C2F200035A829A82DA
S315080050901DE0084490F8370050B940F29451C2F226
S315080050A000010B7040F29553C2F200031A700EE02D
S315080050B00344DBB21846A342A9DB40F29451C2F27C
S315080050C000010B7040F29553C2F200031A7041F6C4
S315080050D0A864C2F200040323637641F62073C2F281
S315080050E0000393F82620227293F82720627293F819
S315080050F02820A27293F82930E3720120FFF7B0FA4C
S3150800510041F69C63C2F2000342221A7000222282F0
S3150800511041F69063C2F200031A8042F26253C2F269
S3150800512000031A8000F096FEBCE041F69C63C2F2CA
S31508005130000320221A7000F08DFE41F6A463C2F225
S3150800514000031B6800225A76ABE441F62073C2F2CC
S31508005150000393F82F3013F0010F38D012F0100F18
S3150800516035D141F6A863C2F200031B8A002B40F032
S315080051704F8241F69064C2F200042088013080B262
S31508005180FFF76EFA41F69C63C2F200031A7842F002
S3150800519010011970238833B141F69C63C2F20003EB
S315080051A042F012021A7000F055FE41F6A864C2F2E7
S315080051B0000401232382082363760023E37641F65D
S315080051C02073C2F20003112283F82F209DE113F009
S315080051D0200F18D041F62073C2F2000393F834006A
S315080051E0000293F8351041F6A063C2F2000340EAC4
S315080051F001051C682C441C6041F69063C2F200034A
S315080052001888411B198041F69063C2F2000318887A
S3150800521060B112F0100F09D141F69C63C2F2000387
S315080052201A7842F002021A70FFF71AFA41F620734A
S31508005230C2F2000393F8302093F8313003EB0223CF
S315080052409BB240F28052C2F20002138041F6A86275
S31508005250C2F20002928A934200D823B940F28053E0
S31508005260C2F200031A8041F6A863C2F2000340F2B4
S315080052708052C2F2000212885A8241F69C63C2F238
S3150800528000031B7813F0030F00F0C28142F2625349
S31508005290C2F2000300221A8000F0DCFD41F6A86481
S315080052A0C2F2000441F69C63C2F200031B7813F0B5
S315080052B0200F0ED042F26253C2F2000300221A8077
S315080052C0627641F62073C2F20003142283F82F2077
S315080052D01BE113F0100F12D042F26253C2F2000320
S315080052E000221A800123238204236376E27641F69C
S315080052F02073C2F20003112283F82F2005E142F23F
S315080053006252C2F200021288DAB113F0010F1CBF12
S315080053100023238201D1218A71B9618A8A4282BF18
S3150800532042F26253C2F20003198042F26253C2F299
S3150800533000031B88238204E042F26253C2F2000390
S3150800534019800023E37641F6A063C2F2000341F612
S315080053509462C2F2000212681A6042F26253C2F202
S3150800536000031B887BB1238A6BB141F69062C2F2B7
S3150800537000022833138041F62073C2F20003182274
S3150800538083F82F20C7E041F69C63C2F200031B781E
S3150800539013F0020F00F03C8141F69063C2F200035D
S315080053A028221A8041F62073C2F20003102283F8DD
S315080053B02F20B0E041F69C63C2F200031B7813F07D
S315080053C0010F00F0258141F6A863C2F2000300220E
S315080053D05A7641F69C63C2F2000310221A7000F056
S315080053E039FD15E141F69063C2F20003188808B149
S315080053F0FFF736F941F62073C2F2000393F82F300F
S3150800540013F0010F1FD041F69C63C2F200031B780C
S3150800541013F0010F41F6A863C2F200031FBF07226B
S315080054205A7600229A7612BF1A8206225A760120E6
S31508005430FFF716F941F69C63C2F2000310221A70B0
S3150800544000F008FD56E041F69C63C2F200031B78A3
S3150800545013F0010F08D041F6A863C2F20003052233
S315080054605A7600221A82D3E041F69063C2F200030C
S315080054701B88002B3ED1CBE041F69063C2F20003B5
S31508005480188808B1FFF7ECF841F62073C2F200035A
S3150800549093F82F3013F0010F13D041F6A863C2F228
S315080054A0000307225A7600229A760120FFF7D8F8D9
S315080054B041F69C63C2F2000310221A7000F0CAFC7F
S315080054C018E041F69063C2F200031B8893B99FE087
S315080054D041F69C63C2F200031B7813F0010F00F03B
S315080054E0978041F6A863C2F2000307225A76002283
S315080054F09A768DE041F62073C2F20003102283F8F3
S315080055002F2041F6A864C2F2000441F69063C2F265
S31508005510000328221A8041F62073C2F200035022A3
S3150800552083F82E20227A41F62073C2F2000383F80C
S315080055302A20627A83F82B20A27A83F82C20E27A32
S3150800554083F82D20227B83F82620627B83F8272088
S31508005550A27B83F82820E27B83F829200622DA75C5
S31508005560A2885A84E2889A8441F61C72C2F2000222
S315080055701188598352889A832288DA8362881A8422
S31508005580637E13F0100F41F62073C2F200031DBFAD
S31508005590002283F8312083F83020062202BF83F8E0
S315080055A030200A2283F8312041F62074C2F2000422
S315080055B04023A37541F69063C2F200031B881A0ABA
S315080055C022746374002584F8355084F8345065864F
S315080055D0FFF770F8C04360864523A373E5736575C6
S315080055E0257540F28253C2F200031A88013292B23C
S315080055F01A80130AA374E2742583FFF749F8C04397
S31508005600208341F69C63C2F2000300221A7038BD5B
S3150800561041F69063C2F2000300221A8041F69C63A9
S31508005620C2F200031A7038BD40F29453C2F2000366
S3150800563001211970FFF7B6BA40F29453C2F200037B
S3150800564001221A70E4E700BF030A43EA002080B289
S31508005650704700BF10B504460A1E0FDD42F26253BA
S31508005660C2F200031A8041F69463C2F20003186876
S31508005670844203D0214692B201F012FF10BD00BF4A
S315080056802DE9F00340F29653C2F200034FF0000CE6
S3150800569083F800C040F29855C2F200052B46012255
S315080056A01F461C88CCB15E88BEB1B0F80080A04504
S315080056B013D14488B44210D140F29653C2F2000383
S315080056C083F800C0086878608B883B8140F2F953FC
S315080056D0C2F200031B78BB725AE0541CE4B20C33C6
S315080056E0092C02D094462246DAE72B4600221E46AB
S315080056F01C884CB95C883CB940F29653C2F2000348
S315080057001A70082A36D104E00132D2B20C33082ABC
S31508005710EDD1002340F2F952C2F200021678B046E3
S315080057201F4699465FFA83FCAA7AC2EB0804BC4274
S31508005730C2BFC2EB0602E146D7B201330C35082BCD
S31508005740F0D140F29753C2F200031F7040F2F853AB
S31508005750C2F2000383F8009040F29653C2F20003A7
S3150800576083F8009040F29853C2F2000309EB490906
S3150800577003EB89060268334643F8042B0A6872600D
S315080057808A889A8040F2F953C2F200031B78B372F2
S31508005790BDE8F003704700BFF0B440F2F953C2F217
S315080057A000031E780136F6B21E7040F29853C2F214
S315080057B000030122002740F29654C2F200045888DA
S315080057C01988014389B259B1997A711A772907DD7F
S315080057D0194601F8017B5F70013101F8017B0F70F2
S315080057E022700132D2B20C33092AE8D1F0BC7047D4
S315080057F038B541F69063C2F200031B88292B06D8F8
S3150800580041F69063C2F2000300221A8038BD41F6C1
S315080058109063C2F2000300221A8041F62073C2F296
S3150800582000039B8AB3F5807F03D0B3F5007F59D078
S3150800583038BD41F62072C2F2000241F61C73C2F26C
S315080058400003D28C1B889A4269D141F62072C2F2B3
S31508005850000241F61C73C2F20003128D5B889A425D
S315080058605DD12F4CA51F20462946FFF709FFA4F155
S315080058701C03002204F8082C022204F8072C54F80A
S31508005880062C626034F8022C228140F28C52C2F255
S315080058900002106844F8060C928824F8022C44F892
S315080058A0160C24F8122C626844F81C2C228924F859
S315080058B0182C9A8B62816288A28141F61C72C2F208
S315080058C000021188998352886280082204F8102CF5
S315080058D0062204F80F2C41F69063C2F200032A222E
S315080058E01A8038BD41F62072C2F2000241F61C73D6
S315080058F0C2F20003D28C1B889A4210D141F620725C
S31508005900C2F2000241F61C73C2F20003128D5B88D4
S315080059109A4204D1024908460639FFF7B1FE38BD56
S315080059203C1F002038B541F62073C2F20003D98B1C
S315080059308AB24FF6FF739A4215D141F62073C2F226
S315080059400003188C4FF6FF7398420CD141F620736A
S31508005950C2F2000347F69032C0F6000210681860DB
S3150800596092889A80ADE041F61C73C2F200031B8848
S315080059705A4041F61873C2F200031B881A4212D124
S3150800598041F62073C2F200031A8C90B241F61C73DA
S31508005990C2F200035B88584041F61873C2F200034E
S315080059A05B8818420CD040F2FC53C2F2000341F661
S315080059B01472C2F200021188198052885A8005E0D2
S315080059C040F2FC53C2F2000319805A8040F2FC539D
S315080059D0C2F2000318885D8840F29853C2F20003A9
S315080059E000221C46198881420AD15988A94207D142
S315080059F040F29653C2F200031A70082A58D109E0F9
S31508005A000132D2B20C33082AEBD140F29653C2F2D5
S31508005A1000031A7041F62074C2F200042046FF21E2
S31508005A20062201F091FD002384F8203084F8213005
S31508005A3084F8223084F8233084F8243084F825301A
S31508005A4040F28C52C2F200021168C4F8061092881D
S31508005A506281C4F81610628340F2FC52C2F2000258
S31508005A601188E1845288228541F61C72C2F200022E
S31508005A701188A1835288E283237501226275A37374
S31508005A80E2730822227463740623A3740423E3745E
S31508005A9022730623637341F6A063C2F20003363409
S31508005AA01C6041F69063C2F200032A221A8038BDB0
S31508005AB041F62073C2F2000354F8040F1860A28856
S31508005AC09A8041F62073C2F2000340F28C52C2F269
S31508005AD000021168C3F8061092885A8108221A73C0
S31508005AE000225A7341F69063C2F200031A880E32F6
S31508005AF01A8038BD08B500F00DFC01F05FFC01F016
S31508005B0043FC00F08BFC00F00FF800F0F1FB08BD39
S31508005B1008B500F001FC01F06DFC00F0BDFD00F0D9
S31508005B2029F800F0BDFB08BD30B583B0FF238DF81A
S31508005B30043000258DF8055000F0D0F900F0FAFF82
S31508005B4040F21804C2F200040123237001F07CFB22
S31508005B50257000F09DF80323237040F20063C2F21B
S31508005B6000031B78DBB2012B02D101A800F0D6F99D
S31508005B7003B030BD08B540F20460C2F2000001F07F
S31508005B80E1F801280BD140F21803C2F20003012202
S31508005B901A7040F20460C2F2000000F0BFF940F249
S31508005BA00460C2F2000001F0A3FB01280BD140F209
S31508005BB01803C2F2000300221A7040F20460C2F20F
S31508005BC0000000F0ABF940F20460C2F2000000F0F9
S31508005BD0BBF801280BD140F21803C2F200030322D6
S31508005BE01A7040F20460C2F2000000F097F908BD8E
S31508005BF0704700BF38B505460C4640F21803C2F296
S31508005C0000031B78012B02D1C9B201F047F840F214
S31508005C101803C2F200031B781BB92846E1B201F04B
S31508005C2033FB40F21803C2F200031B78032B03D19F
S31508005C302846E1B200F066F800F068F938BD00BF02
S31508005C4040F21803C2F200031878012804D002288B
S31508005C5014BF4020002070470820704740F2180300
S31508005C60C2F200031878012804D0022814BF402085
S31508005C70002070470820704740F20063C2F2000314
S31508005C8001221A70704700BF08B500F035F908BD43
S31508005C9008B5FBF795FF01F0BFFB40F24863C2F277
S31508005CA0000300F5FA70186001F0B6FB40F2446391
S31508005CB0C2F2000300F51C5010301860FEF700FD14
S31508005CC041F61C73C2F200034FF6A9621A8043F626
S31508005CD01371598041F61873C2F200034FF6FF712B
S31508005CE019800021598041F61473C2F200031A8004
S31508005CF040F213125A804EF60300FEF7FBFCFCF73F
S31508005D0073F808BDF8B541F6A463C2F200031F682C
S31508005D10FB693B628E4659B14E1EB6B20136002368
S31508005D2007F11C05C45CEA1814720133B342F9D1B1
S31508005D300EF10401A7F8641007F12000FFF78AFCAA
S31508005D40FB690133FB61F8BD10B5FCF75FF8002865
S31508005D503ED041F69062C2F20002108041F62073EE
S31508005D60C2F200039C894FF40060FFF76DFC844281
S31508005D7013D10120FEF7D8FC41F69063C2F2000366
S31508005D801B882BB3FFF7CEFDFCF768F841F6906346
S31508005D90C2F2000300221A801AE041F62073C2F20A
S31508005DA000039C8940F60600FFF74EFC84420FD19B
S31508005DB0FFF71EFD41F69063C2F200031B883BB154
S31508005DC0FCF74CF841F69063C2F2000300221A80F1
S31508005DD001F022FB40F24863C2F200031B689842B6
S31508005DE022D340F24862C2F2000203F5FA73136046
S31508005DF041F6A463C2F2000341F6A862C2F20002A9
S31508005E001A600220FEF790FC41F69063C2F2000386
S31508005E101B884BB1FFF786FDFCF720F841F6906327
S31508005E20C2F2000300221A8001F0F6FA40F2446337
S31508005E30C2F200031B68984209D340F24462C2F2D8
S31508005E40000203F51C5310331360FFF7A5FC00206E
S31508005E5010BD00BF10B541F6A463C2F200031C686A
S31508005E6041F69C63C2F200031B7813F0400F05D07D
S31508005E700123E3610023A4F8643010BD13F0010F79
S31508005E801CBF0022A4F8642013F0040F06D0B4F84F
S31508005E90641019B104F12000FFF7DCFB41F69C639E
S31508005EA0C2F200031B7813F0020F0AD00023A4F8ED
S31508005EB0643041F6A063C2F200031868043000F0AB
S31508005EC02DF810BD40F24C63C2F20003FE22DA70D0
S31508005ED018710222A3F84420704700BF40F24C63B1
S31508005EE0C2F2000300221A709A6483F84320A3F8CA
S31508005EF044209A705A70704740F24C63C2F200030D
S31508005F001878003018BF0120704700BF40F24C6374
S31508005F10C2F20003002283F84320704738B50446CE
S31508005F200178FF2923D100F08FFA18B91020FFF75E
S31508005F30C9FF96E140F24C64C2F200040023637084
S31508005F4001252570FF22E270102222716371FFF786
S31508005F5077FEA071FFF782FEE071FFF77FFE000A69
S31508005F6020726572A5720823A4F8443079E140F2DC
S31508005F704C63C2F200031B78012B40F09081C939AB
S31508005F80352900F26B81DFE811F0DB006901690150
S31508005F906501690169015901FC0042012F01690186
S31508005FA06901690169016901690169016901690193
S31508005FB06901690169016901690169016901690183
S31508005FC06901690169016901690169016901690173
S31508005FD069016901690169016901690169017F004E
S31508005FE0540036007300690169016901A10069015D
S31508005FF0B900BD00CE004578FFF722FE013885427C
S3150800600003DD2220FFF75EFF2BE140F24C65C2F26A
S315080060100005281DA96C627800F0F0FEFF23EB70DE
S315080060206278AB6C1344AB6463780133A5F84430EB
S3150800603017E14578FFF704FE0138854203DD222083
S31508006040FFF740FF0DE1616840F24C65C2F20005BA
S31508006050A964281D627800F0D1FEFF23EB706278F0
S31508006060AB6C1344AB6463780133A5F84430F8E0AD
S3150800607040F24C63C2F20003FF22DA7042689A6467
S315080060800122A3F84420ECE040F24C63C2F200037C
S31508006090FF22DA709B6C406840B11844002213F85E
S315080060A0011B0A44D2B28342F9D100E0002240F231
S315080060B04C63C2F20003C3F8072001221A710022BA
S315080060C05A719A710822A3F84420CAE040F24C6338
S315080060D0C2F20003FF22DA7047F69832C0F60002D1
S315080060E09A6400221A715A719A710721D9711A7223
S315080060F05A729A720822A3F84420B2E00020FFF7E9
S31508006100E1FEAEE040F24C63C2F20003FF22DA7011
S3150800611000221A71597859719A71DA711A7206221F
S31508006120A3F844209DE040F24C63C2F2000300222B
S315080061301A705A70FF22DA700122A3F8442090E000
S3150800614040F24C63C2F200039D6CFFF779FD411ED5
S315080061502846621C01F01CF918B93120FFF7B2FE77
S315080061607FE040F24C64C2F20004FF23E370A56CA2
S31508006170FFF766FD013D2844A0640123A4F84430D6
S315080061806FE04578FFF75CFD0238854203DD222083
S31508006190FFF798FE65E040F24C63C2F20003FF2267
S315080061A0DA700122A3F84420617839B901F0FCF8C5
S315080061B0002856D13120FFF785FE52E040F24C63A5
S315080061C0C2F20003986CA21C01F0E2F818B931205B
S315080061D0FFF778FE45E040F24C63C2F200036178AF
S315080061E09A6C0A449A643CE040F24C64C2F2000499
S315080061F0FF23E370002525716571FFF721FDA07166
S31508006200E571257265720723A4F8443029E040F247
S315080062104C63C2F20003986C616801F0BDF818B9C6
S315080062203120FFF74FFE1CE040F24C63C2F2000338
S31508006230FF22DA700122A3F8442012E000F0EEFDF6
S3150800624040F24C63C2F20003FF22DA700122A3F87F
S31508006250442006E03120FFF735FE02E02020FFF754
S3150800626031FE40F24C63C2F2000393F84330012B2F
S3150800627002D11020FFF726FE40F24C63C2F200035B
S31508006280B3F844100BB2002B09DD40F24C60C2F2A1
S315080062900000012380F843300330FFF7ABFC38BD1C
S315080062A008B5FFF7F1FC012820D000F0CDF8E8B1D9
S315080062B040F29863C2F200031B78012B16D101F055
S315080062C0ABF840F29C63C2F200031B6803F51C534B
S315080062D0103398420AD340F29863C2F200030022B0
S315080062E01A7000F0BBF808B900F070FD08BD00BFD1
S315080062F008B540F29863C2F2000301221A7001F051
S315080063008BF840F29C63C2F200031860FFF7C8FFDF
S3150800631008BD00BF704700BF704700BF00F00F03FD
S31508006320092802D903F13700704703F1300040F21B
S315080063301C03C2F200031B6803445B7803F00303E3
S31508006340022B08BF2038C0B2704700BF38B50546D3
S315080063500C460009FFF7E2FF207005F00F00FFF773
S31508006360DDFF60700023A370204638BD30B40246B6
S3150800637003464CF6CD40CCF6CC400131A0FB034396
S31508006380DB08FAD1002301F801394CF6CD45CCF6E5
S31508006390CC450846A5FB0243DB0803EB8304A2EBC6
S315080063A04402303201F801291A46002BF1D130BCDB
S315080063B0704700BFF0B440F21C03C2F200031F6826
S315080063C000231C46C15C7A18527802F00302022A9E
S315080063D008BF2039C9B2A1F13002D2B2A1F13A05FB
S315080063E0EDB2162A94BF00260126062D8CBF354627
S315080063F046F0010565B9092A84BFA1F13702D2B270
S315080064002401E4B22244D4B20133022BDAD101E0EA
S31508006410002000E02046F0BC704700BF08B540F2F7
S31508006420E063C2F200030020187040F2EC61C2F289
S315080064300001FDF7BBFB30B147F6A030C0F60000FF
S315080064407C2100F069FB08BD40F2E063C2F200035C
S315080064501878D0F1010038BF0020704708B5FFF75B
S3150800646013FC01280FD040F2E063C2F200031B7848
S315080064705BB9F9F7C5FE012809D140F2E063C2F21B
S315080064800003187008BD002008BD002008BD0020C4
S3150800649008BD00BF027840F21C03C2F200031B6865
S315080064A09918497801F00301022908BF203A532AAE
S315080064B00ED1407803445B7813F0040F0AD03128D4
S315080064C00AD032280AD0332814BF03200220704786
S315080064D0032070470320704700207047012070474B
S315080064E070B504460230FFF765FF064605460434D4
S315080064F02046FFF75FFF3044C6B2013DADB2023415
S31508006500012DF5D82046FFF755FFF643F6B2864229
S3150800651014BF0020012070BD2DE9F04115460F4635
S315080065200446002918BF002807D147F6A030C0F650
S31508006530000040F2362100F0EFFA2046FFF7AAFFE6
S315080065400646032808BF002000F0A2802046FFF771
S31508006550C7FF002800F08C80012E29D016B1022E24
S3150800656053D088E0A01CFFF725FF8046201DFFF7C3
S3150800657021FF06023E60A01DFFF71CFF304438606D
S3150800658004F10806A8F103081FFA88F84046002D0A
S315080065907ED00FFA88F7002F6FDD00243046FFF70C
S315080065A009FF285502360134A4B2BC42F6DB66E080
S315080065B0A01CFFF7FFFE8046201DFFF7FBFE060422
S315080065C03E60A01DFFF7F6FE06EB00263E6004F1CE
S315080065D00800FFF7EFFE3044386004F10A06A8F118
S315080065E004081FFA88F84046002D51D00FFA88F79C
S315080065F0002F46DD00243046FFF7DCFE285502361C
S315080066000134A4B2BC42F6DB3DE0A01CFFF7D2FE83
S315080066108046201DFFF7CEFE06063E60A01DFFF74A
S31508006620C9FE06EB00463E6004F10800FFF7C2FE0D
S3150800663006EB00263E6004F10A00FFF7BBFE304475
S31508006640386004F10C06A8F105081FFA88F84046D8
S31508006650F5B10FFA88F7002F17DD00243046FFF74B
S31508006660A9FE285502360134A4B2BC42F6DB0EE078
S315080066704FF6FF700CE000200AE0404608E040466E
S3150800668006E0404604E0404602E0404600E0404658
S3150800669000B2BDE8F08100BF70B540F2E063C2F217
S315080066A000031B78002B00F03382012B3FD1F9F74A
S315080066B0CFFD47F6B830C0F60000F9F713FE47F6E7
S315080066C0DC30C0F60000F9F70DFEF9F7BBFD014610
S315080066D0BD480122FDF780FA48B147F60440C0F6E6
S315080066E00000F9F7FFFD0120F9F7ECFD70BD47F64C
S315080066F00C40C0F60000F9F7F5FD47F61440C0F661
S315080067000000F9F7EFFD47F63840C0F60000F9F744
S31508006710E9FD40F2E463C2F2000300221A605A60FF
S3150800672040F2E063C2F2000302221A7070BD022B27
S3150800673040F0FD8040F2EC64C2F2000440F64430BA
S31508006740C2F200004FF4807104F50D72FDF76AFE7F
S3150800675094F93A32002B13DA47F60440C0F60000E3
S31508006760F9F7C0FD0220F9F7ADFD04F50D70FDF748
S31508006770FFFC40F2E063C2F2000300221A7070BD0B
S3150800678000B340F64431C2F20001084601F5C07173
S315080067900022FFF7C1FE0546B0F1FF3F12D147F6CA
S315080067A00440C0F60000F9F79DFD0320F9F78AFDBD
S315080067B08548FDF7DDFC40F2E063C2F200030022E3
S315080067C01A7070BD2BB2002B2CDD40F2E463C2F2C6
S315080067D000035B686BB940F2E463C2F2000340F65B
S315080067E04432C2F20002D2F880211A602DB25D60EE
S315080067F018E040F64432C2F20002D2F8801140F2A4
S31508006800E462C2F20002126891423EBF40F2E462BC
S31508006810C2F20002116040F2E462C2F2000203FA18
S3150800682085F3536040F2EC63C2F20003D3F83C22CE
S31508006830D3F840329A4240F06B8163480021FDF755
S31508006840A1FC90B147F60440C0F60000F9F74AFDEE
S315080068500420F9F737FD5C48FDF78AFC40F2E0634F
S31508006860C2F2000300221A7070BD47F60C40C0F64B
S315080068700000F9F737FD47F66840C0F60000F9F75B
S3150800688031FD40F2E465C2F2000540F2A064C2F2AE
S31508006890000468682146FFF769FD2046F9F722FDDE
S315080068A047F67440C0F60000F9F71CFD2E68300E56
S315080068B02146FFF74BFDC6F30740A11CFFF746FD2F
S315080068C0C6F30720211DFFF741FDF0B2A11DFFF712
S315080068D03DFD2046F9F706FD47F61850C0F60000BC
S315080068E0F9F700FD2868696800F056FD90B947F683
S315080068F00440C0F60000F9F7F5FC0520F9F7E2FCBC
S315080069003148FDF735FC40F2E063C2F2000300228D
S315080069101A7070BD47F60C40C0F60000F9F7E2FCA5
S3150800692040F2E063C2F2000303221A7070BD032B23
S3150800693040F0EE8040F2EC64C2F2000440F64430C7
S31508006940C2F200004FF4807104F50D72FDF76AFD7E
S3150800695094F93A32002B13DA47F69040C0F6000055
S31508006960F9F7C0FC0220F9F7ADFC04F50D70FDF748
S31508006970FFFB40F2E063C2F2000300221A7070BD0A
S3150800698020B340F64432C2F20002104602F5C07146
S3150800699002F58072FFF7C0FD0546B0F1FF3F15D13D
S315080069A047F6B440C0F60000F9F79CFC0320F9F757
S315080069B089FC0548FDF7DCFB40F2E063C2F2000300
S315080069C000221A7070BD00BF200900202BB2002BD0
S315080069D059DD47F6D840C0F60000F9F783FC2DB21A
S315080069E040F2A064C2F2000428462146FFF7BEFC26
S315080069F02046F9F777FC47F6E840C0F60000F9F7B5
S31508006A0071FC40F64436C2F2000696F88301214628
S31508006A10FFF79CFC96F88201A11CFFF797FC96F8F5
S31508006A208101211DFFF792FC96F88001A11DFFF751
S31508006A308DFC2046F9F756FC47F61850C0F60000BC
S31508006A40F9F750FCD6F88001294606F5807200F061
S31508006A509FFC90B947F60440C0F60000F9F742FCDF
S31508006A600620F9F72FFC2B48FDF782FB40F2E0637E
S31508006A70C2F2000300221A7070BD47F60C40C0F639
S31508006A800000F9F72FFC40F2EC63C2F20003D3F8DA
S31508006A903C22D3F840329A423AD147F60050C0F623
S31508006AA00000F9F71FFC00F07FFC90B947F6044098
S31508006AB0C0F60000F9F716FC0720F9F703FC15489D
S31508006AC0FDF756FB40F2E063C2F2000300221A709B
S31508006AD070BD47F60C40C0F60000F9F703FC47F610
S31508006AE01C50C0F60000F9F7FDFB0A48FDF740FB0D
S31508006AF047F63450C0F60000F9F7F4FB40F2E063BD
S31508006B00C2F2000300221A70F9F7BAFB00F05EF928
S31508006B1070BD00BF2009002008B540F6C843C2F280
S31508006B200003186040F6CC43C2F200031960FFF771
S31508006B30F3FBFCE72DE9F047002347F68450C0F63F
S31508006B4000004FF4FA744AF2104113F80080C21894
S31508006B5092F801C008EB0C0202FB044291FBF2F921
S31508006B6002FB191636B94D4609F1FF3292B2B2F553
S31508006B70806F03D30233242BE7D187E04746E246EA
S31508006B804FF4D043C4F2000300225A611A6842F453
S31508006B9000421A601B6813F4004F09D04FF4D04422
S31508006BA0C4F20004FFF7B8FB236813F4004FF9D1C9
S31508006BB04FF4D043C4F200031A6822F002021A60A6
S31508006BC01A6842F001021A605B6813F0010F09D1D6
S31508006BD04FF4D044C4F20004FFF79EFB636813F039
S31508006BE0010FF9D0013F0AF1FF36360546EA074795
S31508006BF0013D3D434FF4D043C4F20003DD611A68FA
S31508006C0022F001021A605B6813F0010F09D04FF4F5
S31508006C10D044C4F20004FFF77FFB636813F0010F4A
S31508006C20F9D14FF4C843C4F20003D3F8002242F066
S31508006C300102C3F80022D3F81C2222F48042C3F8CA
S31508006C401C22D3F80C2242F48042C3F80C220022FC
S31508006C50C3F8B022C3F8B422D3F8042222F480423F
S31508006C60C3F80422D3F8142222F48042C3F814226B
S31508006C70D3F81C2242F48042C3F81C22D3F800221F
S31508006C8022F00102C3F80022BDE8F08747F66050FB
S31508006C90C0F60000F021FFF73FFF71E738B504465C
S31508006CA00D464FF4D043C4F200039B6813F0806F7F
S31508006CB007D147F66050C0F600004FF4A271FFF7FF
S31508006CC02BFF4FF4D043C4F20003D3F8802102F01F
S31508006CD00102C3F88021D3F8802142F07C4242F4B5
S31508006CE00012C3F88021C3F88451E178A27812040F
S31508006CF042EA016221780A43617842EA0122C3F82E
S31508006D008821E179A279120442EA016221790A43CB
S31508006D10617942EA0122C3F88C21D3F8802142F036
S31508006D200102C3F880219B6813F0806F09D14FF4E4
S31508006D30D044C4F20004FFF7EFFAA36813F0806F9B
S31508006D40F9D038BD4FF4D043C4F20003DB6813F022
S31508006D50030F39D04FF4D043C4F20003D3F8B0215F
S31508006D6040F26763B3EB525F18BF002023D14FF49C
S31508006D70D043C4F20003D3F8B8210270D3F8B8217F
S31508006D80120A4270D3F8B821120C8270D3F8B821CF
S31508006D90120EC270D3F8BC210271D3F8BC21120AB4
S31508006DA04271D3F8BC21120C8271D3F8BC311B0E88
S31508006DB0C3710120FFE74FF4D043C4F20003DA6839
S31508006DC042F02002DA6070470020704708B500F0EC
S31508006DD0E7FA90B1FEF70CFF00F004FB00F0F6F9B5
S31508006DE020F0604020F07F004EF60853CEF20003F4
S31508006DF0186000F0EBF94368984708BD70B5561E51
S31508006E00B6B24AB14C1E0E44451A14F8013F2B552A
S31508006E10FFF782FAB442F8D170BD00BF08B500F09A
S31508006E200FFB08BDF8B507460024254647F6D85691
S31508006E30C0F60006FFF770FAA359BB420ED83119FF
S31508006E4049680B449F4209D247F6D853C0F6000357
S31508006E5005EB450203EB8203187AF8BD01350C34BD
S31508006E606C2CE7D1FF20F8BD2DE9F8438046006871
S31508006E70FFF7D8FFFF2830D0FBF720F8F320FBF701
S31508006E803DF8FBF741F801281CBF002408F1040966
S31508006E9004D1FBF729F80020BDE8F883D8F800608C
S31508006EA0A71959F80450FFF737FA38462946FBF769
S31508006EB0A9F8082807D1A359AB4206D10434B4F57A
S31508006EC0007FEBD103E0002402E0002400E0012467
S31508006ED0FBF70AF82046BDE8F8830020BDE8F883EA
S31508006EE038B504460D4640F6D043C2F20003984230
S31508006EF009D04FF44043C0F6000399420BD0FFF780
S31508006F00B3FF20B917E040F6D464C2F20004C5F313
S31508006F10080393B903E040F6D044C2F2000423689C
S31508006F209D420CD0204640F8045B29464FF4007277
S31508006F30FFF764FF03E0002038BD002038BD204677
S31508006F4038BD00BF2DE9F04106460C4617461D46DA
S31508006F504FEA51284FEA48280368B3F1FF3F06D1A4
S31508006F6040F8048B41464FF40072FFF747FF336839
S31508006F70434505D030464146FFF7B2FF0646D0B135
S31508006F803368E41A3444043408F50078FFF7C4F982
S31508006F90331DE31AB3F5007F06D330464146FFF7A3
S31508006FA09FFF064650B1041D17F8013B04F8013B44
S31508006FB0013DEBD105E00020BDE8F0810020BDE8E9
S31508006FC0F0810120BDE8F08140F6D463C2F20003E7
S31508006FD04FF0FF321A6040F6D043C2F200031A603F
S31508006FE0704700BF70B504460D461646FFF71AFFF0
S31508006FF0FF281BD0681E2044FFF714FFFF2817D070
S31508007000620A4FF44043C0F60003B3EB422F07BFB2
S3150800701040F6D040C2F2000040F6D460C2F200004A
S31508007020214632462B46FFF78DFF70BD002070BD06
S31508007030002070BDF8B505460E46FFF7F3FE044678
S31508007040701E2844FFF7EEFE0546FF2C18BFFF28E2
S3150800705033D084422BD8022C2BD90B282BD8FAF7FD
S315080070602DFFF320FAF74AFFFAF74EFF01281EBF55
S3150800707047F6A856C0F60006022703D1FAF734FFEA
S315080070800020F8BDFFF748F936F814003946FAF734
S3150800709081FF082803D0FAF727FF0020F8BD01343E
S315080070A0E4B2A542EED2FAF71FFF0120F8BD002090
S315080070B0F8BD0020F8BD0020F8BD0020F8BD00BFCF
S315080070C000B583B040F6D043C2F200031B68B3F1A3
S315080070D0FF3F08BF01201CD040F6D043C2F2000390
S315080070E099685A681144DA6811441A6911445A6948
S315080070F011449A690A44D96953185B4202AA42F8AC
S31508007100043D4CF28810C0F600000421FFF76AFF20
S31508007110FFE703B05DF804FB4CF20402C0F6000278
S315080071204FF44043C0F6000310681B6818444CF23D
S315080071300803C0F600031B6818444CF20C03C0F69B
S3150800714000031B6818444CF21003C0F600031B68C2
S3150800715018444CF21403C0F600031B6818444CF29A
S315080071601803C0F600031B6818444CF28813C0F6CF
S3150800717000031B681844D0F1010038BF002070478F
S3150800718008B540F6D043C2F200031B68B3F1FF3FCF
S3150800719006D040F6D040C2F20000FFF765FE88B17F
S315080071A040F6D463C2F200031B68B3F1FF3F0BD06D
S315080071B040F6D460C2F20000FFF756FE003018BF52
S315080071C0012008BD002008BD012008BD4FF440403D
S315080071D0C0F60000704700BF38B504464FF4A0500B
S315080071E0C4F201008021FBF783F990B14FF4A05057
S315080071F0C4F201002146FBF773F94FF4A054C4F218
S315080072000104802520462946FBF772F90028F9D0A3
S3150800721001E0002038BD012038BD00BF10B5044686
S315080072204FF4A050C4F201002021FBF761F90128B0
S3150800723008D14FF4A050C4F20100FBF755F92070AD
S31508007240012010BD002010BD10B584B04FF4614375
S3150800725000930023ADF80430ADF80630ADF80830D9
S31508007260ADF80C300C23ADF80A304FF4A054C4F234
S31508007270010420466946FBF7B5F820460121FBF7CD
S3150800728021F904B010BD00BF2DE9F04106460C46B1
S31508007290402906D947F64460C0F600007721FFF773
S315080072A03BFC2046FFF798FF012806D047F64460C6
S315080072B0C0F600007B21FFF72FFC2546ACB1002461
S315080072C047F64467C0F600074FF08408FFF724F82E
S315080072D0305DFFF781FF012803D038464146FFF7A6
S315080072E01BFC0134A3B2AB42F0D3BDE8F08100BF6A
S315080072F010B5044641F21D13C2F200031B78A3B968
S3150800730041F2D800C2F20000FFF788FF012832D107
S3150800731041F21D13C2F2000301221A7041F21C1336
S31508007320C2F200030020187010BD41F21C13C2F20D
S3150800733000031878134B1844FFF770FF01281CD177
S3150800734041F21C13C2F200031A780132D2B21A7043
S3150800735041F2D803C2F200031B7893420FD12046AC
S315080073600849FFF74BFD41F21D13C2F20003002244
S315080073701A70012010BD002010BD002010BD00208D
S3150800738010BD00BFD910002008B5FFF71DFE08BDC7
S3150800739008B5FFF727FE08BD08B5FFF74BFE08BD81
S315080073A008B5FFF7B9FE08BD08B5FFF789FE10B1A5
S315080073B0FFF7E6FE08BD002008BD00BF4EF2100329
S315080073C0CEF2000300221A6049F23F01C0F2020120
S315080073D059609A600521196041F22013C2F2000330
S315080073E01A6070474EF21003CEF2000300221A60AC
S315080073F0704700BF4EF21003CEF200031B6813F469
S31508007400803F1FBF41F22013C2F200031A680132FF
S3150800741018BF1A60704700BF08B5FFF7EBFF41F2C7
S315080074202013C2F20003186808BD00BF08B547F666
S315080074306860C0F600003621FFF76EFB08BD00BF86
S3150800744010B572B640F20002C2F2000240F2200302
S31508007450C2F200039A4210D2131D0E4CE41A24F00D
S31508007460030404340023104647F69871C0F6000159
S315080074705A581A500433A342FAD1074807494FF01D
S3150800748000028842B8BF40F8042BFADBF8F75AFF27
S3150800749010BD00BF230000208000002064250020C6
S315080074A00F2AF0B445D940EA01039B0745D1A2F15A
S315080074B010070C4603463F0900EB071610362568E9
S315080074C01033103443F8105C54F80C5C43F80C5C29
S315080074D054F8085C43F8085C54F8045C43F8045C08
S315080074E0B342ECD17B1C02F00F0CBCF1030F4FEA40
S315080074F003131944034422D90E461D46644656F81A
S31508007500047B043C032C45F8047BF8D8ACF104044E
S3150800751002F0030224F0030404342344214432B164
S315080075200A4411F8014B914203F8014BF9D1F0BC1A
S3150800753070470346002AF3D1F9E70346F0E76246A7
S31508007540002AEDD1F3E700BF8307F0B448D0541EF4
S31508007550002A43D0CDB2034602E0002C3ED01446A2
S3150800756003F8015B13F0030F04F1FF32F5D1032C86
S315080075702DD9CDB20F2C45EA052545EA054518D97A
S31508007580A4F1100703F110061A463F0906EB071681
S315080075901560103242F80C5C42F8085C42F8045C4C
S315080075A0B242F5D104F00F040137032C03EB07139D
S315080075B00DD91E462246043A46F8045B032AFAD831
S315080075C0221F04F0030422F00302043213442CB1F0
S315080075D0C9B21C4403F8011BA342FBD1F0BC704797
S315080075E014460346C3E700BF2F64656D6F70726F5C
S315080075F0675F6F6C696D65785F73746D3332653478
S3150800760030372E73726563002F626F6F746C6F6705
S315080076102E747874000000002E2F6C69622F75692D
S31508007620702F6E65746465762E630000222A3A3CD4
S315080076303E3F7C7F000000002B2C3B3D5B5D00003D
S31508007640809A90418E418F804545454949498E8F9C
S315080076509092924F994F555559999A9B9C9D9E9FEA
S3150800766041494F55A5A5A6A7A8A9AAABAC21AEAF77
S31508007670B0B1B2B3B4B5B6B7B8B9BABBBCBDBEBF84
S31508007680C0C1C2C3C4C5C6C7C8C9CACBCCCDCECF74
S31508007690D0D1D2D3D4D5D6D7D8D9DADBDCDDDEDF64
S315080076A0E0E1E2E3E4E5E6E7E8E9EAEBECEDEEEF54
S315080076B0F0F1F2F3F4F5F6F7F8F9FAFBFCFDFEFF44
S315080076C001030507090E10121416181C1E000000E7
S315080076D06100620063006400650066006700680078
S315080076E069006A006B006C006D006E006F00700028
S315080076F071007200730074007500760077007800D8
S3150800770079007A00A100A200A300A500AC00AF0092
S31508007710E000E100E200E300E400E500E600E7003F
S31508007720E800E900EA00EB00EC00ED00EE00EF00EF
S31508007730F000F100F200F300F400F500F600F8009E
S31508007740F900FA00FB00FC00FD00FE00FF00010145
S3150800775003010501070109010B010D010F011101C3
S3150800776013011501170119011B011D011F01210133
S3150800777023012501270129012B012D012F013101A3
S315080077803301350137013A013C013E01400142010E
S315080077904401460148014B014D014F015101530176
S315080077A05501570159015B015D015F0161016301E3
S315080077B06501670169016B016D016F017101730153
S315080077C0750177017A017C017E019201B103B2034A
S315080077D0B303B403B503B603B703B803B903BA03CF
S315080077E0BB03BC03BD03BE03BF03C003C103C3037E
S315080077F0C403C503C603C703C803C903CA033004C1
S3150800780031043204330434043504360437043804A6
S3150800781039043A043B043C043D043E043F04400456
S315080078204104420443044404450446044704480406
S3150800783049044A044B044C044D044E044F045104B5
S31508007840520453045404550456045704580459045E
S315080078505A045B045C045E045F0470217121722182
S3150800786073217421752176217721782179217A214E
S315080078707B217C217D217E217F2141FF42FF43FF21
S3150800788044FF45FF46FF47FF48FF49FF4AFF4BFFB6
S315080078904CFF4DFF4EFF4FFF50FF51FF52FF53FF66
S315080078A054FF55FF56FF57FF58FF59FF5AFF000070
S315080078B0C700FC00E900E200E400E000E500E7009C
S315080078C0EA00EB00E800EF00EE00EC00C400C5009B
S315080078D0C900E600C600F400F600F200FB00F90055
S315080078E0FF00D600DC00A200A300A500A720920195
S315080078F0E100ED00F300FA00F100D100AA00BA0099
S31508007900BF001023AC00BD00BC00A100AB00BB004B
S31508007910912592259325022524256125622556253C
S3150800792055256325512557255D255C255B2510259D
S31508007930142534252C251C2500253C255E255F2588
S315080079405A25542569256625602550256C25672501
S3150800795068256425652559255825522553256B25FF
S315080079606A2518250C25882584258C2590258025AB
S31508007970B103DF009303C003A303C303B500C40325
S31508007980A6039803A903B4031E22C603B503292236
S315080079906122B1006522642220232123F7004822B0
S315080079A0B0001922B7001A227F20B200A025A00035
S315080079B04100420043004400450046004700480095
S315080079C049004A004B004C004D004E004F00500045
S315080079D051005200530054005500560057005800F5
S315080079E059005A002100E0FFE1FFE5FFE2FFE3FF4F
S315080079F0C000C100C200C300C400C500C600C7005D
S31508007A00C800C900CA00CB00CC00CD00CE00CF000C
S31508007A10D000D100D200D300D400D500D600D800BB
S31508007A20D900DA00DB00DC00DD00DE0078010001A9
S31508007A3002010401060108010A010C010E011001E8
S31508007A4012011401160118011A011C011E01200158
S31508007A5022012401260128012A012C012E013001C8
S31508007A6032013401360139013B013D013F01410133
S31508007A704301450147014A014C014E01500152019B
S31508007A805401560158015A015C015E016001620108
S31508007A906401660168016A016C016E017001720178
S31508007AA07401760179017B017D01910191039203AD
S31508007AB093039403950396039703980399039A03EC
S31508007AC09B039C039D039E039F03A003A103A3039B
S31508007AD0A403A503A603A703A803A903AA031004DE
S31508007AE011041204130414041504160417041804C4
S31508007AF019041A041B041C041D041E041F04200474
S31508007B002104220423042404250426042704280423
S31508007B1029042A042B042C042D042E042F04010402
S31508007B2002040304040405040604070408040904FB
S31508007B300A040B040C040E040F046021612162215F
S31508007B4063216421652166216721682169216A21EB
S31508007B506B216C216D216E216F2121FF22FF23FFEE
S31508007B6024FF25FF26FF27FF28FF29FF2AFF2BFFD3
S31508007B702CFF2DFF2EFF2FFF30FF31FF32FF33FF83
S31508007B8034FF35FF36FF37FF38FF39FF3AFF00006D
S31508007B90FFFFFFFFFFFF00004F70656E424C540069
S31508007BA02E2E2F2E2E2F2E2E2F536F757263652F86
S31508007BB066696C652E6300004669726D7761726549
S31508007BC020757064617465207265717565737420BB
S31508007BD064657465637465640A0D00004F70656EAC
S31508007BE0696E67206669726D776172652066696C71
S31508007BF06520666F722072656164696E672E2E2E27
S31508007C00000000004552524F520A0D004F4B0A0D14
S31508007C10000000005374617274696E6720746865A9
S31508007C202070726F6772616D6D696E67207365711A
S31508007C3075656E63650A0D0050617273696E67201B
S31508007C406669726D776172652066696C6520746F06
S31508007C50206F627461696E2065726173652073694D
S31508007C607A652E2E2E00000045726173696E6720B4
S31508007C70000000002062797465732066726F6D20BB
S31508007C806D656D6F72792061742030780000000090
S31508007C9052656164696E67206C696E652066726FED
S31508007CA06D2066696C652E2E2E4552524F520A0D6E
S31508007CB000000000496E76616C696420636865633C
S31508007CC06B73756D20666F756E642E2E2E45525237
S31508007CD04F520A0D0000000050726F6772616D6D99
S31508007CE0696E67200000000020627974657320744D
S31508007CF06F206D656D6F7279206174203078000091
S31508007D0057726974696E672070726F6772616D2049
S31508007D10636865636B73756D2E2E2E00436C6F73E7
S31508007D20696E67206669726D776172652066696C2F
S31508007D30650A0D004669726D776172652075706413
S31508007D40617465207375636365737366756C6C79A6
S31508007D5020636F6D706C657465640A0D0000000021
S31508007D602E2E2F2E2E2F2E2E2F536F757263652FC4
S31508007D7041524D434D345F53544D33322F63616E38
S31508007D802E6300000502060206030703080309031B
S31508007D9009040A040B040C040C050D050E050F0551
S31508007DA00F0610061007100800000800100018003B
S31508007DB020002800300038004000480050005800D5
S31508007DC08000880090009800A000A800B000B800C5
S31508007DD0C000C800D000D80000C00008004000005D
S31508007DE00300000000000108000001000400000074
S31508007DF00000020800000200050000000000040858
S31508007E00000002000600000000000608000002004C
S31508007E100700000000000808000002000800000033
S31508007E2000000A08000002000900000000000C0813
S31508007E30000002000A00000000000E080000020010
S31508007E400B0000002E2E2F2E2E2F2E2E2F536F7541
S31508007E507263652F41524D434D345F53544D33324F
S31508007E602F756172742E63002E2E2F2E2E2F2E2E16
S31508007E702F536F757263652F41524D434D345F53CF
S31508007E80544D33322F4743432F766563746F7273AD
S31508007E902E630000002020202020202020202828D3
S31508007EA028282820202020202020202020202020AC
S31508007EB020202020208810101010101010101010EC
S31508007EC0101010101004040404040404040404101C
S31508007ED010101010101041414141414101010101AA
S31508007EE00101010101010101010101010101010174
S31508007EF01010101010104242424242420202020280
S31508007F000202020202020202020202020202020243
S31508007F1010101010200000000000000000000000F3
S31508007F200000000000000000000000000000000043
S31508007F300000000000000000000000000000000033
S31508007F400000000000000000000000000000000023
S31508007F500000000000000000000000000000000013
S31508007F600000000000000000000000000000000003
S31508007F7000000000000000000000000000000000F3
S31508007F8000000000000000000000000000000000E3
S30D08007F900000000000000000DB
S31508007F9801000000010000000000000001020304BF
S31508007FA8010203040607080904000000947E000875
S70508000000F2
